:1068EC00011F00000501013C0200000301FA040035
:1068FC00FA0500030A0A5A0B001E0C00FA0D0003DD
:10690C000E00040F0164100096120132130AFA14DF
:10691C00010215000017010A1801FA1905321A01B3
:10692C000A1B01FA1C05321FFFFF20FFFF23011E6B
:10693C002400642A00FA2B00FA2C50782D003D2EEE
:10694C0000462F001E300064325078330000343281
:10695C00FA350164360164370150380A643C00642E
:10696C003E003C3F000140FFFF411450420A5A4395
:10697C000AC84405324500B44600FA47013C4802B7
:10698C00024C00FA4EFFFF500A0A510596520A3289
:10699C00530B46540A9656020257054658000259A4
:1069AC000A465A32FA5B010A5C0A325E000A5F0040
:1069BC00FE61FFFF64021C66000167FFFF6A0A3C70
:1069CC006B00006C32967300007400007801327911
:1069DC0001327E00FE7FFFFF80FFFF8100008400FC
:1069EC00FE8500AF8600018700FA8901088A000045
:1069FC009900009D0A969E00019FFFFFA0FFFFFAE1
:106A0C00FAFA0065006F00790083008D009700A1F1
:106A1C0000AC00B600C000CA00D400DE00E800F2F2
:106A2C0000580060006800700078008000880090BA
:106A3C00009800A000A800B000B800C100C800D0A9
:106A4C0000D800DF00E600EE00F600410047004DE4
:106A5C0000530059005F0065006C00710077007DE9
:106A6C0000830089008F0095009B00A200A700AC5A
:106A7C0000B200B900C000C500CA00D200D500DDCC
:066A8C0000E100E700EF4D
:103A39009007CAE0FEA3E0FF9068EE126BCBE49317
:103A4900F5999068ECE493FC740193FDEFB50507D3
:103A5900EEB50403754D009007CA126BB22275A723
:103A69001085F97385FA747E017F00E574126BA4E1
:103A7900E5732FFF50010E8E5A8F5B90001FE0FCFB
:103A8900A3E0FDEF2DFDEE3CFC8C5C8D5D22E55D38
:103A9900F5FBE55CF5FCD29322E55DF5E9E55CF51E
:103AA900EAD29422E55DF5EBE55CF5ECD29122E5ED
:103AB9005DF5EDE55CF5EED29222E55DF5FDE55C9F
:103AC900F5FED28722AE5AAF5B74068E048F05FFCE
:103AD900126B948C5C8D5DAE5AAF5B74068E048F4D
:103AE90005FF126BBF8C5A8D5BE55B455A601374F9
:103AF90006C3955BFFE4955AFE8E5A8F5B785C127C
:103B09006BF8E573A85CB80015D3955D4010E573B3
:103B1900C3955DFFE4955CFE8E5C8F5D8010E57357
:103B2900243CC3955DFFE4955CFE8E5C8F5DAE5CC5
:103B3900AF5D743B6F4E6006743C6F4E701AAE5C9D
:103B4900AF5D743B6F4E7005757301800375730229
:103B5900755D3A755C0080037573002290009AE0E8
:103B6900B40104C20E8002D20E90009BE0B401049D
:103B7900C20F8002D20F9000D8E075F0DCA4FFAE2E
:103B8900F0740A8E048F05FF126B949007C0ECF055
:103B9900A3EDF0A20B401674038C068D07126BA4DB
:103BA90074011200399007BEEEF0A3EFF07E017F99
:103BB90000900096E0126BA49000D9E08E048F0566
:103BC900FF126B94740AFF126B948D609000E2E00F
:103BD90075F0DCA4FFAEF0740A8E048F05FF126B3A
:103BE900949007C4ECF0A3EDF09000E4E06013902A
:103BF90000E4E0F5F0741684FF7E00EF9007D2F040
:103C0900800674649007D2F09000DAE090007FF0AB
:103C1900900124E0900069F09000B3E090006BF00F
:103C29009000DCE090006CF0900088E090006DF06E
:103C39009000CEE090006EF090010EE0900072F0DE
:103C4900900172E0900073F0900173E0900074F0BD
:103C5900900174E0900075F0A228B34016900172AB
:103C6900E0700C900173E07006900174E0600280CE
:103C790002C22874E390007EF09000C3E0B40B0800
:103C890074E390007EF0805A9000C3E0B41912905A
:103C990000D9E09069F912008CE49390007EF080DD
:103CA900419000C3E0B41E129000D9E0906A171247
:103CB900008CE49390007EF080289000C3E0B42843
:103CC900129000D9E0906A4112008CE49390007E32
:103CD900F0800F9000C3E0B446089000BAE090006D
:103CE9007EF09000F3E0FE9000C1E06E600A900063
:103CF900C1E09000F3F0D227900082E0FE9000C06E
:103D0900E0B50627900084E0FE9000DEE0B5061BD2
:103D1900900083E0FE9000ECE0B5060F900085E08E
:103D2900FE900093E06E7003023E40740890010F0C
:103D3900F0900093E0B4010674009000F9F090004F
:103D490093E0B4020674009000DEF0900093E0B4B2
:103D5900030674009000EBF09000DEE0D39401407C
:103D690014741A900111F074009006D4F074009044
:103D790006D5F0800C7400900111F0741A9006D4E5
:103D8900F09000C0E0601474069000A7F0740090F1
:103D990006D8F074009006D9F0800C74009000A742
:103DA900F074069006D8F09000C0E0B402147407CD
:103DB9009000A8F074009006DCF074009006DDF025
:103DC900800C74009000A8F074079006DCF0900055
:103DD900ECE0B40114741B900112F074009006E435
:103DE900F074009006E5F0800C7400900112F074F4
:103DF9001B9006E4F0D2279000C0E0900082F0907A
:103E090000ECE0900083F09000DEE0900084F090F8
:103E19000093E0900085F0900093E090006AF090A4
:103E290000ECE090006FF09000C0E0900070F0901E
:103E390000DEE0900071F09000F6E0B40117900008
:103E49002B740FF0A374FFF090002DE4F0A3F0742D
:103E5900029000F6F09000F6E0B4034190002DE0E6
:103E6900FEA3E0FF90002BE0FCA3E0FD126BF074D1
:103E790010126BA47408120039EF90007BF0EF70F8
:103E89000674FF90007BF074009000F6F090002C0F
:103E9900E090007CF090002BE090007DF09000878E
:103EA900E0900043F0900043E0240C900044F0902F
:103EB9000043E02418900045F0900043E02424904A
:103EC9000046F0900043E02430900047F090004411
:103ED900E0D3943C400B900044E0C3943C900044F0
:103EE900F0900045E0D3943C400B900045E0C3942A
:103EF9003C900045F0900046E0D3943C400B900084
:103F090046E0C3943C900046F0900047E0D3943CCF
:103F1900400B900047E0C3943C900047F090004D5F
:103F2900E4F0900043E0643B6007900043E0B43C58
:103F390020900043E0B43B06740290004DF09000DD
:103F490043E0B43C0690004D7401F09000437401C5
:103F5900F090004EE4F0900044E0643B600790006C
:103F690044E0B43C20900044E0B43B067402900065
:103F79004EF0900044E0B43C0690004E7401F0907D
:103F890000447401F090004FE4F0900045E0643B78
:103F99006007900045E0B43C20900045E0B43B0642
:103FA900740290004FF0900045E0B43C0690004F39
:103FB9007401F09000457401F0900050E4F0900015
:103FC90046E0643B6007900046E0B43C2090004620
:103FD900E0B43B067402900050F0900046E0B43C17
:103FE900069000507401F09000467401F090005161
:103FF900E4F0900047E0643B6007900047E0B43C80
:1040090020900047E0B43B067402900051F0900004
:1040190047E0B43C069000517401F09000477401E8
:10402900F0900087E0FE9000EAE02E900053F090B7
:1040390000C5E0B40173900053E075F00C84AFF053
:104049007E00EF4E7006900053E004F0900053E0BC
:104059000475F00C84AFF07E00EF4E7006900053AB
:10406900E014F0900048E0B43D069000487401F077
:10407900900053E0D3943C400B900053E0C3943C30
:10408900900053F0900053E0D3941E400D900053DC
:10409900E0C3941E900054F0800A900053E0241E5F
:1040A900900054F075511E8041900053E075F00C5A
:1040B90084AFF07E00EF4E7006900053E004F0905C
:1040C9000053E00475F00C84AFF07E00EF4E7006EB
:1040D900900053E014F0900053E075F00C84AFF0B9
:1040E9007E00EF900053F075510C9000CDE09000E8
:1040F90048F0900048E075F00C84AFF07E00EF4E78
:104109007006900048E004F0900048E00475F00C57
:1041190084AFF07E00EF4E7006900048E014F090F6
:104129000048E0B43D069000487401F0900048E072
:10413900240C900049F0900048E0241890004AF0BF
:10414900900048E0242490004BF0900048E024308F
:1041590090004CF0900049E0D3943C400B9000490A
:10416900E0C3943C900049F090004AE0D3943C406D
:104179000B90004AE0C3943C90004AF090004BE059
:10418900D3943C400B90004BE0C3943C90004BF01F
:1041990090004CE0D3943C400B90004CE0C3943C1D
:1041A90090004CF022C293C294C291C292C287C2BB
:1041B90090E5B554EFF5B5E5B554DFF5B5C296C24E
:1041C90095C2A0C297C2A2C2A1E5B554BFF5B5E593
:1041D900B5547FF5B5E5B554FBF5B5C210755E4626
:1041E9009000D0E07005756D028003756D037555FB
:1041F9000075540090001474FFF0A374DCF0C2162B
:10420900C218C21AC21CC21E74C890002FF074C80A
:10421900900033F074C8900037F074C890003BF0F8
:1042290074C890003FF0755300755200C20B754673
:1042390000E56FB40903756F00756300900021E410
:10424900F0A3F0757010C213C214C2159007C0E034
:10425900FEA3E0FF7403126BA474011200399007E6
:10426900BEEEF0A3EFF0C20275570075560090003C
:1042790018E4F0A3F0C2297559007558009000920E
:10428900E075F032A4FDACF0900029ECF0A3EDF05C
:10429900C239A22DB39205A22EB39206A22FB392D0
:1042A90007A230B39208A231B39209A232B3920A9B
:1042B9002275A71085F97385FA747E017F00E5746C
:1042C900126BA4E5732FFF50010E8E5A8F5BAC5C05
:1042D900AD5DEF2DFDEE3CFC8C5C8D5DD293D294EF
:1042E900D291D292D287E55DF5FBE55CF5FCE55DFF
:1042F900F5E9E55CF5EAE55DF5EBE55CF5ECE55D31
:10430900F5EDE55CF5EEE55DF5FDE55CF5FE75A71A
:10431900002285F97385FA747E017F00E574126BBA
:10432900A4E5732FFF50010E8E5A8F5B7E017F76B5
:1043390090010BE0126BA4AC5AAD5BED2FFFEC3E84
:10434900FE8E5C8F5DE55DF5EDE55CF5EE90007F39
:10435900E4F07412900056F02285F97385FA747EA0
:10436900017F00E574126BA4E5732FFF50010E8ED7
:104379005A8F5B9007C0E0FCA3E0FDEF2DFDEE3CFA
:10438900FC8C5C8D5DE55DF5FDE55CF5FE22056463
:1043990022A2DBB340089000DAE090007FF0A2D8B7
:1043A900400AC296C295C2A0C297C2A275D840223D
:1043B90085A77275A710A2D8B34002C293A2D9B338
:1043C9004002C294A2DAB34002C291A2DBB3400216
:1043D900C292A2DCB34002C28775D8408572A72277
:1043E900900047E4936406600280FE74C89007C693
:1043F900F8E4F0E8A3F075B50075840175A70075B8
:10440900FFA0900052E4F075C91075A70F75A1C7F8
:1044190075A70075D90075CE0C75A70F75F1FE75D6
:10442900F2FF75F30775F47875A4BA75A5FF75A63B
:104439000775AE0075AFFF75D48175D5FF75D6FFC9
:1044490075D7FF75A70075A20175A14775F809759C
:10445900D80075D90475DD0975DE0975D84075A7C9
:104469001075D80075D90475DA0975DB0975DC0989
:1044790075DD0975DE0975D84075A70075E60875FB
:10448900E71075BC0175BE0475BD6C75BE0775BDB9
:10449900A075BE0875BD0175BC0075BB1875BC203B
:1044A90075BA0875E88075D11375A70F75E105759B
:1044B900E20075C7401241AE759700759780740A7E
:1044C900126B847597C0E5975420700280F8758F38
:1044D9000275A700D2AF75980075A90C75A70F755D
:1044E900AB4375ADFB75AC1E75A71075C91875CAB8
:1044F9000075CB0075C80475A700758912758E04FF
:10450900758C00758A00C2A9D28C758D00758B00D7
:10451900D2ABD28E75EF0675D944C2997509C875A3
:1045290008001200E975B5001204E974639007C622
:10453900F8E4F0E8A3F012037574C89007C6F8E42C
:10454900F0E8A3F07509647508001200E990006AA3
:10455900E0900093F0900093E0D39403400C740032
:10456900900093F0740090006AF0C222900093E0EA
:104579009064F7F82828738028A2B44002D22280D8
:104589002075A70F75F30F75A700A2A34002D222C9
:10459900800F75A70F75F31775A700A2A44002D263
:0145A90022EF
:0C64F70002458002458202458A02459B56
:1045AA00A222B3405E757308E573D3940E501FE5DB
:1045BA00739007C6F8E4F0E8A3F0120244750964A0
:1045CA007508001200E97873740126F650DA74024D
:1045DA009000CFF090006AE0900093F0900093E092
:1045EA00906503F8282873801674009000F9F0800B
:0F45FA000E74009000DEF0800674009000EBF06D
:0C6503000245F10245F30245FB0246038D
:10460900D221805C757301E573D39407501FE5735C
:104619009007C6F8E4F0E8A3F0120244750964753E
:1046290008001200E97873740126F650DA740190D3
:1046390000CFF090006AE0900093F0900093E09032
:10464900650FF8282873801674009000F9F0800E21
:0E46590074009000DEF0800674009000EBF01C
:0C650F0002464F02465102465902466106
:10466700C221900069E0900124F090006AE0900078
:1046770093F090006BE09000B3F090006CE0900036
:10468700DCF090006DE0900088F090006EE0900004
:10469700CEF090006FE09000ECF0900070E090009A
:1046A700C0F0900071E09000DEF0900072E09001A1
:1046B7000EF0900073E0900172F0900074E09001AA
:1046C70073F0900075E0900174F0900172E0700C47
:1046D700900173E07006900174E060028004C228C4
:1046E7008002D2289000D9E07006740A9000D9F0B1
:1046F7009000BAE0700674E39000BAF09000C0E052
:1047070004900082F09000C1E09000F3F0123B6546
:10471700E5B54401F5B57406900058F074019000B2
:1047270059F0740390005BF0740590005CF074110D
:1047370090005DF0740690005EF0740190005FF0E9
:104747007400900064F07400900067F074FF9000AC
:1047570068F0743690015DF0743090015EF0742D4E
:1047670090015FF07432900160F07420900161F065
:104777007431900162F07430900163F074439001DA
:1047870064F07479900165F0746C900166F07420A0
:10479700900167F07420900168F07420900169F02F
:1047A700742090016AF0742090016BF09000F5E09E
:1047B70090007BF09000ACE090007CF09000ADE0C2
:1047C70090007DF0A2B6B3920CA2B3B3920DA2A44F
:1047D700B39224A2B4B39225A2A3B39226900077F2
:1047E700E4F0756F00743A900786F074FD900787C0
:1047F700F0900078E4F09007C0E0FEA3E0FF7403B8
:10480700126BA474011200399007BEEEF0A3EFF00B
:10481700756E01900056E4F0C223756300C211D291
:1048270012C202757100C22BD203C22CD204C22D50
:10483700D205C22ED206C22FD207C230D208C23149
:10484700D209C232D20AC22712009E755F00756B69
:1048570000756100756532756600756700756800DB
:10486700756900756A00900021E4F0A3F0756C008B
:10487700D2B2D2A4D2B0D2B1D2A3D2A7D2A6D2A555
:10488700D2B7900092E0D394FA400674FA9000925F
:10489700F07E017F0090007DE0126BA490007CE029
:1048A7002FFF50010E90002BEEF0A3EFF0EFD39403
:1048B700FFEE940F400790002BE4F0A3F090007BED
:1048C700E0700674FF90007BF09000CFE0D3940275
:1048D700400674019000CFF09000D0E07005756D30
:1048E700028003756D039000D1E0D39401400674F4
:1048F700009000D1F09000D7E0C3940A5006740AE4
:104907009000D7F09000E1E0700674019000E1F0AC
:104917009000E1E0B4FF0674FE9000E1F09000E83B
:10492700E0D394FE400674FE9000E8F090010EE09C
:10493700D394024006740190010EF0900124E0D355
:10494700940140067401900124F074019000EEF088
:1049570074019000EFF074009000F6F0740090017D
:1049670016F074299006CCF0742A9006D0F07408DB
:104977009006E0F0741C9006E8F0D29C9000C1E02D
:10498700D39404400674049000C1F0E570D39410EA
:1049970040037570109006CDE0D3940C4006740068
:1049A7009006CDF09006D1E0D3940C4006740090A9
:1049B70006D1F09006D5E0D3940C4006740090061B
:1049C700D5F09006D9E0D3940C400674009006D930
:1049D700F09006DDE0D3940C400674009006DDF0FD
:1049E7009006E1E0D3940C400674009006E1F09045
:1049F70006E5E0D3940C400674009006E5F09006B7
:104A0700E9E0D3940C400674009006E9F0D2EC7507
:104A1700CF01A298B34005C298120646E54D60063D
:104A2700A299B3B340028005C299120C57E54E64B0
:104A3700016005E54EB4040280D5C28E7E107F006A
:104A4700E564126BA4E58D75F010A4FDACF0EF2DB5
:104A5700FDEE3CFCE58B75F01084FF7E00ED2FFF2B
:104A6700EC3EFE8E548F55D28E9000B3E0600990D5
:104A770000B3E0C3943D40028056900023126BB20E
:104A8700900023E0FEA3E0FF900025E0FCA3E0FDFB
:104A9700EFB5053CEEB50438B220A20BB34013A224
:104AA70020B34008E5B54404F5B58006E5B554FBE9
:104AB700F5B5900025E0FEA3E0FF900027E0FCA3FA
:104AC700E0FDEF2DFDEE3CFC900025ECF0A3EDF0B2
:104AD7009000C0E060099000C0E0C39403400280EA
:104AE7007D122D96A20BB35009900077E0C3942F47
:104AF700400280069000AAE0F545E54575F005A45B
:104B0700FFAEF09007C8EEF0A3EFF0900097E0C378
:104B170095614007E55FC3956050079007C8E4F0CB
:104B2700A3F0AE2EAF2F9007C8E0FCA3E0FDEFD3B4
:104B37009DEE9C4004C290800B900077E0C39446A2
:104B47005002D2909000C0E0B40213A290B3400884
:104B5700E5B554EFF5B58006E5B54410F5B5900019
:104B6700C0E0B4031C122EB1AE2EAF2F9007C8E0E1
:104B7700FCA3E0FDEFD39DEE9C4004D2908002C2DF
:104B870090A2B6300C01B350030251EBA2B6300C21
:104B970001B350030251EBA2B6300E01B35003022A
:104BA700504C756E009000B3E0B43D13A20EB340B5
:104BB70008E5B554FBF5B58006E5B54404F5B5053C
:104BC7005EA210B3B35013AE54AF55900014E0FC7F
:104BD700A3E0FDEDC39FEC9E4003024D04E56DB4D9
:104BE700032EA229B34022E55EB43B03756D01E5B0
:104BF7005EC3943B50069000567401F0E55ED39473
:104C07003B40067402900056F0755E01D229806021
:104C1700E56DB40206756D01755E3BE55EB43B0557
:104C2700755E01804B900056E07036E55EC3943B9D
:104C370050069000567401F0E55ED3943B4006742D
:104C470002900056F0E55EC3943B5002D223E55E26
:104C5700D3943B4002D223C296C295C2A0C297C248
:104C6700A29000D0E0B401051241AE8003755E0149
:104C7700AE56AF57AC54AD55EF2DFDEE3CFC74026C
:104C87008C068D071200398E568F579000B3E0605F
:104C9700099000B3E0C3943D40028043900023E0B5
:104CA700FEA3E0FF9000B3E08E048F05FF126B9424
:104CB70074018C068D07120039900027EEF0A3EFE0
:104CC700F0900027E0F8A3E0900025C8F0A3C8F013
:104CD700900023E4F0A3F0C220E5B554FBF5B5A29C
:104CE700B4B34002C225A2A4B34002C224A2A3B314
:104CF7004002C226A223B34002C223803AAE56AF77
:104D070057AC54AD55EF2DFDEE3CFC74018C068D70
:104D1700071200398E568F57E56DC39402500DACBC
:104D270054AD5574B8C39D740B9C40028009124161
:104D3700AE7406900056F0E55EB43B127403900023
:104D470056F0D2239000D0E0B401031241AEAE5822
:104D5700AF59AC54AD55EF2DFDEE3CFC8C588D5939
:104D6700AE54AF55EFD39DEE9C401190001BE0FA77
:104D7700A3E0FBEBC394E8EA9403400280069000AB
:104D87001B126BB2900018E0FEA3E0FFAC54AD55C8
:104D9700EF2DFDEE3CFC900018ECF0A3EDF0900039
:104DA700D0E0B40118AE54AF557405126BA474016A
:104DB700120039900014EEF0A3EFF08011AE54AF5B
:104DC700557402126BA4900014EEF0A3EFF0C28E9C
:104DD700758D00758B00756400755501755400D28B
:104DE7008EE55E240E75F00F84AFF07E00EF4E70F7
:104DF70075900018E0F8A3E0900016C8F0A3C8F07B
:104E0700900016E0FEA3E0FFEF4E600B7C7D7D690E
:104E1700126A928E528F53900018E4F0A3F0AE52AC
:104E2700AF537428BE00039F5010E5632FFF500156
:104E37000E74011200398E528F538553639000D739
:104E4700E0A852B8000DD395534008E5539000559C
:104E5700F080099000D7E014900055F0E56D6006EA
:104E6700755300755200E55E640B6005E55EB42975
:104E7700099000C0E060031223D29000C5E0B4019E
:104E870014900053E0655E6007900054E0B55E0340
:104E9700756F00801E900053E0655E6013900053AD
:104EA700E02418655E6009900053E02424B55E0392
:104EB700756F00A211B35006A210B3B34003024F9F
:104EC7006D90008CE0B4017390010EE0B4021412EF
:104ED7000E26900080E075F0BEA4FFAEF08E5C8FCA
:104EE7005D8056E56775F00A84FF7E00900586129F
:104EF7006BCBE0F55B755A00AE5AAF5B9000B1E043
:104F0700126BA474648E048F05FF126B948C5C8DF6
:104F17005DE55D90001AF0AE5AAF5B90008AE01233
:104F27006BA474648E048F05FF126B9474BE8C0699
:104F37008D07126BA48E5C8F5D801790008AE075D9
:104F4700F0BEA4FFAEF08E5C8F5D9000B1E09000E4
:104F57001AF0E561C394CC5006E55D455C700280AC
:104F6700031242BAD211E56DB40106E55E64116021
:104F77000280097570019000577401F0E56D6003B8
:104F87000250479000D3E0600D90007FE0A852B830
:104F970000069553400280509000D3E0B4022F9052
:104FA7000043E0655E601F900044E0655E60179017
:104FB7000045E0655E600F900046E0655E60079023
:104FC7000047E0B55E03757003756C00800CC20086
:104FD700756C00900021E4F0A3F090007FE060067C
:104FE7007409900056F08058900043E0B55E0B7549
:104FF70070019000577401F08046900044E0B55E60
:105007000B7570017402900057F08034900045E0F2
:10501700B55E0B7570017403900057F08022900005
:1050270046E0B55E0B7570017404900057F0801070
:10503700900047E0B55E097570017405900057F060
:10504700A20EB3920CA20EB330B601B350030251B5
:10505700EB756E019000B3E0B43D13A20EB34008A8
:10506700E5B54404F5B58006E5B554FBF5B5E5B5FA
:105077004401F5B5742F900077F0A20E920CE55E0F
:10508700D3944A4014D210E55ED39485400B740440
:10509700900056F0D223755E469000DBE0B401071E
:1050A700E56AC39414400280091241AE741390005C
:1050B70056F0A22B300301B35017A22BB34008E5DB
:1050C700B54408F5B58006E5B554F7F5B5A22B92BA
:1050D70003A22C300401B35017A22CB34008E5B546
:1050E7004402F5B58006E5B554FDF5B5A22C92044A
:1050F700A22D300501B3500FA22DB34004D2A180D9
:1051070002C2A1A22D9205A22E300601B3500FA212
:105117002EB34004D2908002C290A22E9206A22FF4
:10512700300701B35017A22FB34008E5B54410F577
:10513700B58006E5B554EFF5B5A22F9207A230303A
:105147000801B35017A230B34008E5B54420F5B5C0
:105157008006E5B554DFF5B5A2309208A2313009D3
:1051670001B35017A231B34008E5B54440F5B58007
:1051770006E5B554BFF5B5A2319209A232300A014E
:10518700B35017A232B34008E5B54480F5B58006A1
:10519700E5B5547FF5B5A232920AE56AC39441504A
:1051A70009740E900056F01241AE90005EE0FE903A
:1051B700005AE0C39E400990005AE0D39408400982
:1051C70074FB900056F01241AE900063E0601590BA
:1051D7000063E0FE90005DE06E600974FE9000568B
:1051E700F01241AEA223B3400AC296C295C2A0C232
:1051F70097C2A290010BE0600CAE52AF537414BE7D
:1052070000059F40028048900093E090651BF828B6
:105217002873803BA2B4B35005A225B34002800592
:1052270012431BD2258028A2A3B35005A226B34060
:1052370002800512431BD2268015A2A4B35005A2F3
:0F52470024B34002800512431BD2248002800052
:10651B0002521902521B02522E02524102525402D3
:02652B005256C6
:10525600A213B3B35008900048E0655E6002803642
:10526600A201B35006A200B3B340028023123A67EC
:10527600123A979000ECE0B40113A202B34008E59D
:10528600B54480F5B58006E5B5547FF5B575A7003C
:10529600C213D214D215A214B3B35008900049E039
:1052A600655E60028036A201B35006A200B3B34029
:1052B600028023123A67123AA29000ECE0B401137E
:1052C600A202B34008E5B54480F5B58006E5B554BD
:1052D6007FF5B575A700D213C214D215A215B3B3C4
:1052E600500890004AE0655E60028036A201B35025
:1052F60006A200B3B340028023123A67123AAD9079
:1053060000ECE0B40113A202B34008E5B54480F511
:10531600B58006E5B5547FF5B575A700D213D2144E
:10532600C215A213B3B3500890004BE0655E60024D
:105336008036A201B35006A200B3B3400280231206
:105346003A67123AB89000ECE0B40113A202B340F7
:1053560008E5B54480F5B58006E5B5547FF5B57525
:10536600A700C213D214D215A214B3B350089000EA
:105376004CE0655E60028036A201B35006A200B31F
:10538600B340028023123A67123AC39000ECE0B4AD
:105396000113A202B34008E5B54480F5B58006E5E1
:1053A600B5547FF5B575A700D213C214D215E570B2
:0E53B60090652DF8282873025A369000C1E049
:06652D000253BD0253C041
:1053C400906560F8282873121EAE8012121EAE80FB
:0E53D4000D121F388008121FE48003121FE420
:0F6560000253CB0253D00253D50253DA0253DF5A
:1053E200757002025A36122110122227A239B340D6
:1053F200229000B5E0F56C900086E0256CFE9000EE
:1054020055E075F01E84FC7F00EE2CF5367410908A
:105412000056F09007BEE0FEA3E0FF740A126BA4F0
:10542200900016E0FCA3E0FD74098F02FF126B945A
:105432008D078C038E048A058B06126A929007C22E
:10544200EEF0A3EFF074F0BE00039F500B74F090E7
:1054520007C2F8E4F0E8A3F0E53670037536019070
:1054620007C2E0FEA3E0FFE5362FFF50010E9007D2
:0D547200C2EEF0A3EFF0757003900057E05C
:036533000253E828
:10547F0090656FF8282873802BA23A400375700A45
:10548F008022A23A400375700B8019A23A4003752F
:10549F00700C8010A23A400375700D8007A23A403D
:0454AF000375700E03
:10656F0002548602548802549102549A0254A30290
:02657F0054AC1A
:1054B300025A369006CDE060031224EA90010CE014
:1054C300B4011490010DE0A852B80004955350079D
:1054D300E55FC39560400280097415900056F002A1
:1054E30055669000C1E0D39402403F900095E024BC
:1054F30003A852B8000495535009900097E0D39540
:105503006150028008D2017408900056F090009513
:10551300E0A852B80005D39553500B900097E024B0
:1055230003C395615002C2018039900095E02403C2
:10553300A852B8000495535007E55FC39560400235
:105543008008D2017408900056F0900095E0A852AC
:10555300B80005D395535009E560240FC3955F50F8
:1055630002C2019000DBE07007E56AC394144002B5
:105573008002D201A2014005757004800A75701083
:10558300900021E4F0A3F0A20BB34029E56775F086
:105593000A84FF7E00900586126BCBE0C3946950AA
:1055A30005122407800F9007C0E0F8A3E09007BE20
:0C55B300C8F0A3C8F0025A369000C1E016
:066536000254B60255BB41
:1055BF00906581F8282873120F108012120F108037
:0E55CF000D1210BE80081211708003121170B0
:0F6581000255C60255CB0255D00255D50255DA48
:1055DD009006D1E060031225C6757005025A361289
:1055ED0012B07570069006D5E060031226B69006CF
:1055FD00D9E06003122792025A3690001AE0600635
:10560D00A20BB3B34002801D90001AE02529FFAE16
:10561D002850010E8E288F29E55ED3940C500690EC
:10562D00001AE014F01214F67570079006DDE060B4
:10563D000312286E9006E1E0600312294A025A36E1
:10564D0090010EE0B40203120E9E1218F57570084B
:10565D009006E5E06003122A269006E9E060031249
:10566D002B02025A36121CB1A213B35005A214B369
:10567D0040028006D213D214D215757010025A361C
:10568D00025A36900031E0C394465008C2967446D3
:10569D00900031F090004DE0B4011DE5362406F583
:1056AD00369007C2E0FEA3E0FF74062FFF50010EF7
:1056BD009007C2EEF0A3EFF090004DE0B4021DE5AF
:1056CD0036240CF5369007C2E0FEA3E0FF740C2FD4
:1056DD00FF50010E9007C2EEF0A3EFF085365B751B
:1056ED005A00900043E0F573123ACEE55D9000311B
:1056FD00F090000AE55AF0A3E55BF0E573900032F7
:10570D00F0C2179007C2E0F55AA3E0F55B90004395
:10571D00E0F573123ACEE55D90002FF0900000E5B4
:10572D005AF0A3E55BF0E573900030F0C216E56D1D
:10573D00B4010575700B8003757003025A36900025
:10574D0035E0C394465008C2957446900035F090EC
:10575D00004EE0B4011DE5362406F5369007C2E093
:10576D00FEA3E0FF74062FFF50010E9007C2EEF06E
:10577D00A3EFF090004EE0B4021DE536240CF53693
:10578D009007C2E0FEA3E0FF740C2FFF50010E90B6
:10579D0007C2EEF0A3EFF085365B755A009000441A
:1057AD00E0F573123ACEE55D900035F090000CE512
:1057BD005AF0A3E55BF0E573900036F0C21990073F
:1057CD00C2E0F55AA3E0F55B900044E0F573123AA0
:1057DD00CEE55D900033F0900002E55AF0A3E55B55
:1057ED00F0E573900034F0C218E56DB401057570E5
:1057FD000C8003757003025A36900039E0C394464D
:10580D005008C2A07446900039F090004FE0B401EA
:10581D001DE5362406F5369007C2E0FEA3E0FF74C1
:10582D00062FFF50010E9007C2EEF0A3EFF090008F
:10583D004FE0B4021DE536240CF5369007C2E0FEAC
:10584D00A3E0FF740C2FFF50010E9007C2EEF0A3E2
:10585D00EFF085365B755A00900045E0F573123A0E
:10586D00CEE55D900039F090000EE55AF0A3E55BB2
:10587D00F0E57390003AF0C21B9007C2E0F55AA311
:10588D00E0F55B900045E0F573123ACEE55D9000D2
:10589D0037F0900004E55AF0A3E55BF0E573900056
:1058AD0038F0C21AE56DB4010575700D8003757081
:1058BD0003025A3690003DE0C394465008C29774D7
:1058CD004690003DF0900050E0B4011DE5362406F1
:1058DD00F5369007C2E0FEA3E0FF74062FFF5001DE
:1058ED000E9007C2EEF0A3EFF0900050E0B4021D51
:1058FD00E536240CF5369007C2E0FEA3E0FF740CEC
:10590D002FFF50010E9007C2EEF0A3EFF085365B2E
:10591D00755A00900046E0F573123ACEE55D9000A1
:10592D003DF0900010E55AF0A3E55BF0E5739000B3
:10593D003EF0C21D9007C2E0F55AA3E0F55B900062
:10594D0046E0F573123ACEE55D90003BF09000060F
:10595D00E55AF0A3E55BF0E57390003CF0C21CE561
:10596D006DB4010575700E8003757003025A369083
:10597D000041E0C394465008C2A27446900041F025
:10598D00900051E0B4011DE5362406F5369007C2AE
:10599D00E0FEA3E0FF74062FFF50010E9007C2EE4C
:1059AD00F0A3EFF0900051E0B4021DE536240CF5A4
:1059BD00369007C2E0FEA3E0FF740C2FFF50010EDE
:1059CD009007C2EEF0A3EFF085365B755A0090009C
:1059DD0047E0F573123ACEE55D900041F09000126C
:1059ED00E55AF0A3E55BF0E573900042F0C21F901D
:1059FD0007C2E0F55AA3E0F55B900047E0F573129E
:105A0D003ACEE55D90003FF0900008E55AF0A3E531
:105A1D005BF0E573900040F0C21EE56DB4010375B7
:095A2D006D007570038002800019
:10653C000255EC02560702564D02567202568D0257
:10654C00569002574B0258060258C102597C025A07
:04655C0034025A3675
:105A360090002FE0B55E028003025AD8A21640728B
:105A4600900000E0FEA3E0FFEF4E6021AE56AF5798
:105A5600900000E0FCA3E0FD12000374068E048FA4
:105A660005FF126B94900000ECF0A3EDF09000306F
:105A7600E0601A900000E0FEA3E0FFAC56AD57EFE1
:105A86002DFDEE3CFC900000ECF0A3EDF090003014
:105A9600E0D39401401A900000E0FEA3E0FFAC566C
:105AA600AD57EF2DFDEE3CFC900000ECF0A3EDF0C1
:105AB600D216AE54AF55900000E0FCA3E0FDEFC354
:105AC6009DEE9C400D124362D296C21674C8900099
:105AD6002FF0A216B3B3500790002FE0B55E0280F8
:105AE6000D124362D29674C890002FF0C216900031
:105AF60031E0B55E028003025B93A217407290000C
:105B06000AE0FEA3E0FFEF4E6021AE56AF579000CD
:105B16000AE0FCA3E0FD12000374068E048F05FF65
:105B2600126B9490000AECF0A3EDF0900032E06066
:105B36001A90000AE0FEA3E0FFAC56AD57EF2DFD2C
:105B4600EE3CFC90000AECF0A3EDF0900032E0D3BE
:105B56009401401A90000AE0FEA3E0FFAC56AD5750
:105B6600EF2DFDEE3CFC90000AECF0A3EDF0D21711
:105B7600AE54AF5590000AE0FCA3E0FDEFC39DEEE6
:105B86009C400AC2967446900031F0C217A217B321
:105B9600B35007900031E0B55E02800AC2967446A3
:105BA600900031F0C217900033E0B55E0280030228
:105BB6005C4EA2184072900002E0FEA3E0FFEF4E9A
:105BC6006021AE56AF57900002E0FCA3E0FD120044
:105BD6000374068E048F05FF126B94900002ECF09E
:105BE600A3EDF0900034E0601A900002E0FEA3E01E
:105BF600FFAC56AD57EF2DFDEE3CFC900002ECF0ED
:105C0600A3EDF0900034E0D39401401A900002E036
:105C1600FEA3E0FFAC56AD57EF2DFDEE3CFC900029
:105C260002ECF0A3EDF0D218AE54AF55900002E0AE
:105C3600FCA3E0FDEFC39DEE9C400D124362D2959E
:105C4600C21874C8900033F0A218B3B3500790007E
:105C560033E0B55E02800D124362D29574C890009F
:105C660033F0C218900035E0B55E028003025D098C
:105C7600A219407290000CE0FEA3E0FFEF4E6021F7
:105C8600AE56AF5790000CE0FCA3E0FD1200037483
:105C9600068E048F05FF126B9490000CECF0A3EDBA
:105CA600F0900036E0601A90000CE0FEA3E0FFAC36
:105CB60056AD57EF2DFDEE3CFC90000CECF0A3ED3D
:105CC600F0900036E0D39401401A90000CE0FEA359
:105CD600E0FFAC56AD57EF2DFDEE3CFC90000CEC12
:105CE600F0A3EDF0D219AE54AF5590000CE0FCA332
:105CF600E0FDEFC39DEE9C400AC2957446900035C8
:105D0600F0C219A219B3B35007900035E0B55E0290
:105D1600800AC2957446900035F0C219900037E0AB
:105D2600B55E028003025DC4A21A4072900004E0D0
:105D3600FEA3E0FFEF4E6021AE56AF57900004E0A1
:105D4600FCA3E0FD12000374068E048F05FF126BA0
:105D560094900004ECF0A3EDF0900038E0601A9007
:105D66000004E0FEA3E0FFAC56AD57EF2DFDEE3C80
:105D7600FC900004ECF0A3EDF0900038E0D3940121
:105D8600401A900004E0FEA3E0FFAC56AD57EF2D9D
:105D9600FDEE3CFC900004ECF0A3EDF0D21AAE54FC
:105DA600AF55900004E0FCA3E0FDEFC39DEE9C40E0
:105DB6000D124362D2A0C21A74C8900037F0A21A1C
:105DC600B3B35007900037E0B55E02800D12436210
:105DD600D2A074C8900037F0C21A900039E0B55EC0
:105DE600028003025E7FA21B407290000EE0FEA3BB
:105DF600E0FFEF4E6021AE56AF5790000EE0FCA3D9
:105E0600E0FD12000374068E048F05FF126B94905A
:105E1600000EECF0A3EDF090003AE0601A90000E50
:105E2600E0FEA3E0FFAC56AD57EF2DFDEE3CFC9037
:105E3600000EECF0A3EDF090003AE0D39401401A86
:105E460090000EE0FEA3E0FFAC56AD57EF2DFDEE41
:105E56003CFC90000EECF0A3EDF0D21BAE54AF5517
:105E660090000EE0FCA3E0FDEFC39DEE9C400AC24D
:105E7600A07446900039F0C21BA21BB3B350079022
:105E86000039E0B55E02800AC2A07446900039F07F
:105E9600C21B90003BE0B55E028003025F3AA21C83
:105EA6004072900006E0FEA3E0FFEF4E6021AE5682
:105EB600AF57900006E0FCA3E0FD12000374068EC7
:105EC600048F05FF126B94900006ECF0A3EDF090A2
:105ED600003CE0601A900006E0FEA3E0FFAC56AD81
:105EE60057EF2DFDEE3CFC900006ECF0A3EDF09094
:105EF600003CE0D39401401A900006E0FEA3E0FFC8
:105F0600AC56AD57EF2DFDEE3CFC900006ECF0A331
:105F1600EDF0D21CAE54AF55900006E0FCA3E0FDB8
:105F2600EFC39DEE9C400D124362D297C21C74C80B
:105F360090003BF0A21CB3B3500790003BE0B55E67
:105F460002800D124362D29774C890003BF0C21CC7
:105F560090003DE0B55E028003025FF5A21D40722F
:105F6600900010E0FEA3E0FFEF4E6021AE56AF5763
:105F7600900010E0FCA3E0FD12000374068E048F6F
:105F860005FF126B94900010ECF0A3EDF090003E2C
:105F9600E0601A900010E0FEA3E0FFAC56AD57EFAC
:105FA6002DFDEE3CFC900010ECF0A3EDF090003ED1
:105FB600E0D39401401A900010E0FEA3E0FFAC5637
:105FC600AD57EF2DFDEE3CFC900010ECF0A3EDF08C
:105FD600D21DAE54AF55900010E0FCA3E0FDEFC318
:105FE6009DEE9C400AC297744690003DF0C21DA2E9
:105FF6001DB3B3500790003DE0B55E02800AC2971C
:10600600744690003DF0C21D90003FE0B55E0280F0
:10601600030260B0A21E4072900008E0FEA3E0FFFB
:10602600EF4E6021AE56AF57900008E0FCA3E0FDAE
:1060360012000374068E048F05FF126B94900008FD
:10604600ECF0A3EDF0900040E0601A900008E0FE4E
:10605600A3E0FFAC56AD57EF2DFDEE3CFC900008DB
:10606600ECF0A3EDF0900040E0D39401401A9000CC
:1060760008E0FEA3E0FFAC56AD57EF2DFDEE3CFC6D
:10608600900008ECF0A3EDF0D21EAE54AF55900090
:1060960008E0FCA3E0FDEFC39DEE9C400D124362B9
:1060A600D2A2C21E74C890003FF0A21EB3B350071E
:1060B60090003FE0B55E02800D124362D2A274C822
:1060C60090003FF0C21E900041E0B55E02800302E0
:1060D600616BA21F4072900012E0FEA3E0FFEF4E3C
:1060E6006021AE56AF57900012E0FCA3E0FD12000F
:1060F6000374068E048F05FF126B94900012ECF069
:10610600A3EDF0900042E0601A900012E0FEA3E0DA
:10611600FFAC56AD57EF2DFDEE3CFC900012ECF0B7
:10612600A3EDF0900042E0D39401401A900012E0F3
:10613600FEA3E0FFAC56AD57EF2DFDEE3CFC900004
:1061460012ECF0A3EDF0D21FAE54AF55900012E062
:10615600FCA3E0FDEFC39DEE9C400AC2A2744690EC
:106166000041F0C21FA21FB3B35007900041E0B533
:106176005E02800AC2A27446900041F0C21F9000DF
:10618600DEE0B4020280030262A0900079E0D395BB
:10619600665064900079E0F4042566FE9000E1E024
:1061A6008E00F5F0E884FF7E008F73EFC3941050E5
:1061B6000CEF8573F0A4FDACF08D7380037573FF4F
:1061C600900079E0D39573400B900079E0C3957306
:1061D600F57180037571009000FCE0D3957140065F
:1061E6009000FCE0F5719000FDE0C39571500690BB
:1061F60000FDE0F5718071900079E0C39566FE9030
:1062060000E1E08E00F5F0E884FF7E008F73EFC3B7
:106216009410500CEF8573F0A4FDACF08D738003E1
:106226007573FF85735B755A00900079E0255BFFF7
:10623600AE5A50010E8E5A8F5B74FFBE0009D39F73
:106246004005855B7180037571FF9000FCE0D39576
:106256007140069000FCE0F5719000FDE0C3957179
:1062660050069000FDE0F571A20BB3B3500D9000FF
:106276007AE0FE9000E9E0D39E5002800A7407900F
:106286000056F0C2A1801375A710E5CDC3957140E5
:1062960004C2A18002D2A175A700E56FC39409507C
:1062A6000AA2EDB34005C2ED123050AE54AF55749C
:1062B60010C39F74279E400C900078E0C3945A4008
:1062C600030264F4A210B340091241AE74069000B2
:1062D60056F0A222B34008E5B54404F5B58006E5BC
:1062E600B554FBF5B5A212B3500EE561D394334015
:1062F60007E561C394CC4002804190010EE0B402F0
:1063060014120E26900080E075F050A4FFAEF08EB9
:106316005C8F5D800F90008AE075F050A4FFAEF0B0
:106326008E5C8F5DE55D455C6011E5B54401F5B5B4
:10633600742F900077F01242BAD212900078E0D310
:1063460094014007E561C3941A40028002C212908C
:1063560006CDE060031224EAA22B300301B35017E6
:10636600A22BB34008E5B54408F5B58006E5B5545B
:10637600F7F5B5A22B92039006D1E060031225C66D
:10638600A22C300401B35017A22CB34008E5B54443
:1063960002F5B58006E5B554FDF5B5A22C9204903C
:1063A60006D5E060031226B6A22D300501B3500FC4
:1063B600A22DB34004D2A18002C2A1A22D920590C3
:1063C60006D9E06003122792A22E300601B3500FC1
:1063D600A22EB34004D2908002C290A22E920690C2
:1063E60006DDE0600312286EA22F300701B35017B6
:1063F600A22FB34008E5B54410F5B58006E5B554BF
:10640600EFF5B5A22F92079006E1E0600312294A44
:10641600A230300801B35017A230B34008E5B544A6
:1064260020F5B58006E5B554DFF5B5A230920890A3
:1064360006E5E06003122A26A231300901B350179F
:10644600A231B34008E5B54440F5B58006E5B5543C
:10645600BFF5B5A23192099006E9E06003122B025E
:10646600A232300A01B35017A232B34008E5B54450
:1064760080F5B58006E5B5547FF5B5A232920A904F
:106486000078E0C3945A5010E56FB409099000787B
:10649600E004F0756F00803BE56FB40903756F008B
:1064A600755500755400758D00758B0075640090E8
:1064B6000077E0C394465008900077E004F0800629
:1064C6007446900077F0900077E0B44606E5B55440
:1064D600FEF5B5900078E0D394014007E56AC394D1
:1064E6004140028009740E900056F01241AE024AF5
:0164F600168F
:106590000000010001400160018001A001C001E094
:1065A00002000300039603B603D603F404000500BB
:1065B0000512052405360548055A056C057E05902B
:1065C00005A805C005DE0600061406280646066E68
:1065D00006AE05CF00FF013F015F017F019F01BFB4
:1065E00001DF01FF02FF039503B503D503F303FFAA
:1065F00004FF05110523053505470559056B057D84
:10660000058F05A705BF05CE05F10613062706452C
:10661000066D06AD06ED05DD0FAA0FA50F9F0F9ABB
:106620000F940F8D0F870F800F780F710F680F6019
:106630000F570F4E0F450F3B0F300F250F1A0F0E40
:106640000F020EF50EE80EDB0ECC0EBE0EAE0E9F48
:106650000E8E0E7D0E6C0E5A0E470E340E200E0C52
:106660000DF70DE20DCB0DB50D9D0D850D6D0D5486
:106670000D3A0D200D050CE90CCE0CB10C940C76E6
:106680000C580C3A0C1B0BFB0BDB0BBB0B9A0B795E
:106690000B570B350B130AF10ACE0AAB0A870A64B3
:1066A0000A400A1C09F809D409B0098C0967094392
:1066B000091F08FB08D608B2088E086A0846082396
:1066C00007FF07DC07B9079607730751072F070D68
:1066D00006EC06CA06AA068906690649062A060ABB
:1066E00005EC05CD05B0059205750558053C05205E
:1066F000050504EA04CF04B5049C0482046904512E
:1067000004390422040B03F403DE03C803B2039D1F
:10671000038903750361034D033B03280316030438
:1067200002F202E102D102C002B002A00291028292
:106730000273026502570249023C022F022202162E
:10674000020901FD01F201E601DB01D001C601BB36
:1067500001B101A7019D0194018B018201790170B2
:1067600001680160015801500148014101390132BD
:10677000012B0125011E01180111010B010500FF6C
:1067800000FA0FA60FA00F990F920F8B0F840F7CAA
:106790000F740F6B0F620F580F4E0F430F380F2CF3
:1067A0000F1F0F120F050EF70EE80ED80EC80EB70A
:1067B0000EA50E930E800E6C0E580E420E2C0E156A
:1067C0000DFD0DE40DCB0DB10D950D790D5D0D3F5A
:1067D0000D200D010CE10CC00C9E0C7C0C590C35ED
:1067E0000C100BEA0BC40B9E0B760B4F0B260AFD0D
:1067F0000AD40AAA0A800A550A2A09FF09D409A854
:10680000097C0950092508F908CD08A10875084A2E
:10681000081E07F307C8079D07730749072006F7F7
:1068200006CE06A6067E06570630060A05E405BF14
:10683000059B057705540532051004EF04CE04AE20
:10684000048F047104530435041903FD03E203C7E4
:1068500003AD0394037B0363034B0334031E03085C
:1068600002F302DE02CA02B602A30291027F026DA7
:10687000025C024C023C022C021D020E020001F2DC
:1068800001E401D701CA01BE01B101A6019A018F3D
:106890000185017A01700166015D0153014A0141E0
:1068A000013901310129012101190112010B0104F2
:1068B00000FD00F700F000EA00E400DE00D900D39C
:1068C00000CE00C900C400BF00BA00B500B100ADE1
:1068D00000A800A400A0009C009900950091008EE3
:0C68E000008A008700840081007E007B9D
:10009E007547009007CAE4F0A3F075310075300083
:1000AE00754D00754E00C236D23774FE9007CCF8EF
:1000BE00E4F0E8A3F074FE9007CEF8E4F0E8A3F0C5
:1000CE0074FE9007D8F0745A9007D9F0745A9007BE
:1000DE00DAF0D238C22AC23AC23522750B00750A3E
:1000EE0000AE0AAF0BAC08AD09EDC39FEC9E4016F7
:1000FE0074FF126B8475CF01780B740126F65004D1
:10010E0018E436F650DB22900052E0B4AA1C900799
:10011E0086E0B43C159007C6E0FEA3E0FFEF4E600C
:10012E0009741EBE0004D39F5003020243755D0086
:10013E00755C0075F8099007C6E0FEA3E0FF740732
:10014E006F4E6006740E6F4E7006743A900786F00E
:10015E009007C6E0FEA3E0FF7408BE001ED39F40CA
:10016E001A7E017F089007C6E0FCA3E0FD1DBDFFCF
:10017E00011C1200038E5A8F5B801F9007C6E0FE93
:10018E00A3E0FF7408126BE88F048E057E017F08D2
:10019E00CDCCCD1200038E5A8F5BAE5CAF5D740C6E
:1001AE00D39F74019E500302023EA2F9B3407EE536
:1001BE005D455C700375A382AE5CAF5D74016F4EDE
:1001CE00700375A300AE5CAF5D74026F4E700D9040
:1001DE0007C7E075F002A4FDACF08DA3AE5CAF5D79
:1001EE0074036F4E700375A300AE5CAF5D7403BEF7
:1001FE0000039F5013AC5AAD5BED2FFFEC3EFE900B
:10020E000082126BCBE0F5A3AE5CAF5DEFB40B09D1
:10021E00EEB401057414126B84AE5CAF5DEFB40BDB
:10022E0007EEB4010375F80D785C126BF80201A8A5
:10023E00900052E4F022755D00755C0075F809902F
:10024E0007C6E0FEA3E0FF7408BE001ED39F401A4F
:10025E007E017F089007C6E0FCA3E0FD1DBDFF01F7
:10026E001C1200038E5A8F5B801F9007C6E0FEA300
:10027E00E0FF7408126BE88F048E057E017F08CDB7
:10028E00CCCD1200038E5A8F5BAE5CAF5D7411D372
:10029E009F74019E5003020374A2F9B3500302032C
:1002AE0071E55D455C700375A3D2AE5CAF5D740104
:1002BE006F4E700375A300AE5CAF5D74026F4E702F
:1002CE000D9007C7E075F002A4FDACF08DA3AE5CF7
:1002DE00AF5D74036F4E700375A300AE5CAF5D74BB
:1002EE00046F4E700375A300AE5CAF5D74056F4E68
:1002FE00700375A300AE5CAF5D74066F4E70037530
:10030E00A300AE5CAF5D74076F4E700375A300AEB5
:10031E005CAF5D74086F4E700375A300AE5CAF5D8D
:10032E007408BE00039F5016AC5AAD5BED2FFFEC68
:10033E003EFE90007D126BCBE5A3F075A300AE5C84
:10034E00AF5DEFB41009EEB401057414126B84AEF8
:10035E005CAF5DEFB41007EEB4010375F80D785C79
:10036E00126BF802029722755D00755C0075F80934
:10037E00AE5CAF5D7417BE0004D39F500302044DF4
:10038E00A2F9B3500302044AE55D455C700375A300
:10039E00D2AE5CAF5D74016F4E700375A300AE5CA0
:1003AE00AF5D74026F4E700D9007C7E075F002A43A
:1003BE00FDACF08DA3AE5CAF5D74036F4E70037534
:1003CE00A300AE5CAF5D74046F4E700375A300AEF8
:1003DE005CAF5D74056F4E700375A300AE5CAF5DD0
:1003EE0074066F4E700375A300AE5CAF5D74076F3D
:1003FE004E700375A300AE5CAF5D74086F4E700354
:10040E0075A300AE5CAF5D7408BE00039F500C90E8
:10041E000060126BCBE5A3F075A300AE5CAF5D740C
:10042E00166F4E70057414126B84AE5CAF5D74164D
:10043E006F4E700375F80D785C126BF802037E2216
:10044E00900052E0B4AB0280030204E8755D0075C3
:10045E005C0075F809AE5CAF5D7412BE007CD39F74
:10046E004078A2F9B34070E55D455C700375A382D8
:10047E00AE5CAF5D74016F4E700375A300AE5CAFE2
:10048E005D74026F4E700D9007C7E075F002A4FD0B
:10049E00ACF08DA3AE5CAF5D74036F4E700375A3AD
:1004AE0000AE5CAF5D7403BE00039F500990006503
:1004BE00126BCBE0F5A3AE5CAF5D74116F4E7005A1
:1004CE007414126B84AE5CAF5D74116F4E70037555
:1004DE00F80D785C126BF8020463229007D5E4F0F5
:1004EE0074649007C6F8E4F0E8A3F012037574C8BC
:1004FE009007C6F8E4F0E8A3F074FF900060F07483
:10050E00FF900061F074FF900062F0740090005A4A
:10051E00F074FF900063F07400900065F074019029
:10052E000066F090006CE0B4371A900069E090001D
:10053E0060F090006AE0900061F090006BE0900037
:10054E0062F080469007D57401F074659007C6F886
:10055E00E4F0E8A3F012037574C89007C6F8E4F04F
:10056E00E8A3F090006CE0B4371A900069E09000B8
:10057E0060F090006AE0900061F090006BE09000F7
:10058E0062F0800674029007D5F09007D6E4F074FE
:10059E00669007C6F8E4F0E8A3F012037574C890ED
:1005AE0007C6F8E4F0E8A3F090006BE0B4371290C1
:1005BE000069E090005AF090006AE0900063F080CD
:1005CE00769007D67401F074679007C6F8E4F0E8E9
:1005DE00A3F012037574C89007C6F8E4F0E8A3F010
:1005EE0090006BE0B43712900069E090005AF090E2
:1005FE00006AE0900063F0803E74029007D6F074BB
:10060E00689007C6F8E4F0E8A3F012037574C8907A
:10061E0007C6F8E4F0E8A3F090006BE0B437129050
:10062E000069E090005AF090006AE0900063F0805C
:10063E000674039007D6F022E54E64046006E59931
:10064E0064FF60028031A2364004D2368027E54E28
:10065E00600874E6254E900056F0E54D600874F083
:10066E00254D900056F0E54EB4010280FE754E0009
:10067E00754D00C2368002C236E54E90384AF828D3
:10068E002873754E00E599B4FF03754D01E599B4D5
:10069E00FE03754D02E599B4FD03754D03E599B45E
:1006AE00FC03754D04E599B4FA03754D05E599B44F
:1006BE00FB06754E011241AEE599B4F906754E046E
:1006CE001241AEE599D394E54007E599C394F04005
:1006DE0002801685994F754E027E017F00E54FC34D
:1006EE0094E6126BA48E328F339007CAE4F0A3F017
:1006FE00E599D394C44007E599C394E64002802857
:10070E0085994F754E0374E5C3954FF533753200D9
:10071E00AE32AF33906590126B73E493F87401931D
:10072E009007CAC8F0A3C8F0D299020C569000697F
:10073E00E07005A228B3400280429007CAE0FEA3F3
:10074E00E0FF74FFBE00039F5009EFC39446EE9482
:10075E000640119007CAE0FEA3E0FFEFD3946DEEC2
:10076E00940640139007CAE0FEA3E0FF90008612A5
:10077E006BCBE599F0800385997480119007CAE0E0
:10078E00FEA3E0FF900086126BCBE599F09007CAAE
:10079E00126BB29007CAE0FEA3E0FFEFB40106EEC3
:1007AE00B4070280030209FD900786E0B43C028084
:1007BE00030209FDA22850030208E8C29C900069BA
:1007CE00E0900124F090006AE0900093F090006BAE
:1007DE00E09000B3F090006CE09000DCF090006DC3
:1007EE00E0900088F090006EE09000CEF090006FE8
:1007FE00E09000ECF0900070E09000C0F09000717E
:10080E00E09000DEF0900072E090010EF090007328
:10081E00E0900172F0900074E0900173F09000751A
:10082E00E0900174F0123B6590007BE09000F5F0D3
:10083E0090007CE09000ACF090007DE09000ADF078
:10084E0074639007C6F8E4F0E8A3F074AB9000521E
:10085E00F012044E900052E4F07464F5097508002D
:10086E001200E9A2214039757301E573D394075044
:10087E002DE5739007C6F8E4F0E8A3F074AA900093
:10088E0052F0120115E573C39407500A7464F5090A
:10089E007508001200E97873740126F650CC803783
:1008AE00757308E573D3940E502DE5739007C6F853
:1008BE00E4F0E8A3F074AA900052F0120115E5736B
:1008CE00C3940E500A7464F5097508001200E97895
:1008DE0073740126F650CC0209E7C29C900124E005
:1008EE00900069F0900093E090006AF09000B3E001
:1008FE0090006BF09000DCE090006CF0900088E0CF
:10090E0090006DF09000CEE090006EF09000ECE064
:10091E0090006FF09000C0E0900070F09000DEE06C
:10092E00900071F090010EE0900072F07400900053
:10093E0073F07400900074F07400900075F074639E
:10094E009007C6F8E4F0E8A3F074AB900052F012F2
:10095E00044E900052E4F07464F50975080012001C
:10096E00E9757301E573D394075026E5739007C6B6
:10097E00F8E4F0E8A3F074AA900052F01201157496
:10098E0064F5097508001200E97873740126F650B3
:10099E00D3D29C7599FB743C900786F0757308E56D
:1009AE0073D3940E5026E5739007C6F8E4F0E8A3CF
:1009BE00F074AA900052F01201157464F5097508CE
:1009CE00001200E97873740126F650D374C89007AC
:1009DE00C6F8E4F0E8A3F080FE74C89007C6F8E409
:1009EE00F0E8A3F0D29C754E00754D007599FB0290
:1009FE000C569007CAE0FEA3E0FFEF4E70068599F5
:100A0E00317530009007CAE0FEA3E0FF74016F4E0F
:100A1E00701BAC30AD31AA32AB33ED2BFBEC3AFA96
:100A2E008A068B07900086126BCBE599F09007CA69
:100A3E00126BB29007CAE0FEA3E0FF74026F4E7015
:100A4E0021AC30AD3174566D4C7006E54F64E660E6
:100A5E000280031241AE123B65854F99754E0075AB
:100A6E004D00020C569007CAE0FEA3E0FF900086F0
:100A7E00126BCBE599F09007CA126BB29007CAE0E1
:100A8E00FEA3E0FFAC32AD338F028E038C068D07D2
:100A9E009065D4126B73E493F9740193FEEAD39EBE
:100AAE00EB994009854F99754E00754D00020C5615
:100ABE009007CAE0FEA3E0FF900086126BCBE5998B
:100ACE00F09007CA126BB29007CAE0FEA3E0FFEFE8
:100ADE00B40006EEB401028003020C56900062E0F0
:100AEE00D394C7400B900062E0C394C8F550801AAF
:100AFE00900062E0D39463400B900062E0C3946474
:100B0E00F5508006900062E0F550E55075F002A4B5
:100B1E00FFAEF08F73EF900086126BD6EFFCE0FD08
:100B2E00EC900089126BD6EDFCE0FDEC2DB5500279
:100B3E008003020C470FEF900086126BD6E573FF11
:100B4E00E0FCEF90008A126BD6ECFFE0FCEFC39C4A
:100B5E00B550028003020C47E573900088126BD6E5
:100B6E00E573FFE0FCEF90008B126BD6ECFFE0FC20
:100B7E00EF2CB550028003020C47E57390008C12E7
:100B8E006BD6E0C39550900069F0E57390008D121E
:100B9E006BD6E0C3955090006AF0E57390008E120C
:100BAE006BD6E0C3955090006BF0740090006CF023
:100BBE0074FF90006DF0E573900090126BD6E0C359
:100BCE00955090006EF0E573900091126BD6E0C3D5
:100BDE00955090006FF0E573900092126BD6E0C3C3
:100BEE009550900070F0E57390008F126BD6E0C3B5
:100BFE0095509007C6F8E4F0E8A3F074AB9000525D
:100C0E00F012044E7464F5097508001200E990079D
:100C1E00C6126BB212044E7464F509750800120008
:100C2E00E99007C6126BB212044E7599F97464F509
:100C3E00097508001200E980FE7599FF7464F509C4
:080C4E007508001200E980FEA8
:0F384A0002069002073B020A00020A73020ABE3E
:100C560022E54D903859F8282873020D699007CA85
:100C6600E0FEA3E0FF900058126BCBE0F5999007E9
:100C7600CA126BB29007CAE0FEA3E0FF74116F4E72
:100C86007003754D00020D69856E99020D69900716
:100C9600CAE0FEA3E0FF900086126BCBE0F599EF69
:100CA600B40107EEB40703754D009007CA126BB284
:070CB600020D699007CBE07D
:0F385900020C60020C63020C8E020C94020CB97C
:100CBD00903A0CF8282873855399020D5E855F993B
:100CCD00020D5E856199020D5E856599020D5E8549
:100CDD006799807D85689980788569998073856A23
:100CED0099806E900022E0F5998066A237B3400797
:100CFD007599FAC2378041A227B3400575990F80C7
:100D0D00359007D5E0600A9007D5E024DCF5998091
:100D1D00169007D6E0600A9007D6E024DEF599809C
:100D2D0006900056E0F599900056E4F09007D5E452
:100D3D00F09007D6E4F0C2278017856B9980128555
:100D4D006699800D856C9980087599FC8003754DA9
:010D5D000095
:103A0C00020CC4020CCA020CD0020CD6020CDC0252
:103A1C000CE1020CE6020CEB020CF0020CF8020DAD
:0D3A2C0047020D4C020D51020D56020D5BBC
:0B0D5E009007CA126BB28003123A39F2
:03386800020D66E8
:100D690022E537255BFFAE5A50010E900086126BC3
:100D7900CBE0F538E537255BFFAE5A50010E0FBFC2
:100D890000010E900086126BCBE0F539853F3BE5FB
:100D990038B539058538378041E539D39538401D4F
:100DA900E539C39538853AF0A4FFAEF0E53B8E04EA
:100DB9008F05FF126B94ED2538F537801DE538C393
:100DC9009539853AF0A4FFAEF0E53B8E048F05FF17
:100DD900126B94EDF4042538F53722E539D39538AB
:100DE900401DE539C39538853AF0A4FFAEF0E53BDF
:100DF9008E048F05FF126B94ED2538F537801DE5BC
:100E090038C39539853AF0A4FFAEF0E53B8E048FDF
:100E190005FF126B94EDF4042538F5372290008C08
:100E2900E0B40170E56775F00A84FF7E008F37E54D
:100E39006775F00A84ADF07C008D3A753F0A755AE2
:100E490005755B24E537C394115005120D6A8006B8
:100E59009005BBE0F537E537900080F0E56775F060
:100E69000A84FF7E008F37E56775F00A84ADF07C50
:100E7900008D3A753F0A755A05755B5AE537C39473
:100E8900115005120D6A80069005F1E0F537E53736
:100E990090001AF02290008CE0B4016AE56775F0C1
:100EA9000A84FF7E008F37E56775F00A84ADF07C10
:100EB900008D3A753F0A755A05755B36E537C39457
:100EC900115005120D6A80069005CDE0F53785377A
:100ED9004BE56775F00A84FF7E008F37E56775F08B
:100EE9000A84ADF07C008D3A753F0A755A05755B29
:100EF90048E537C394115005120D6A80069005DF45
:100F0900E0F53785374C22E55F75F00484FF7E00F4
:100F19008F37E55F75F00484ADF07C008D3A753F3D
:100F290004755A01755B00E537C3943F5005120DEE
:100F39006A80069001C5E0F5378537297528009044
:100F49000055E075F020A4FFAEF09000D7E08E04C4
:100F59008F05FF126B948D379000BFE0D3955F50DA
:100F6900030210169000E3E0D3955F4010ED900165
:100F7900C6126BD6E0F52B752A000210139000AE4D
:100F8900E0D3955F4043E5379001C6126BD6E0F593
:100F990038E5379001E6126BD6E0F5399000E3E0C9
:100FA900F404255FF53A9000AEE0FE9000E3E0F42A
:100FB900042EF53BE538B539058538378003120D20
:100FC900E485372B752A008041E5379001E6126BDD
:100FD900D6E0F538E537900206126BD6E0F5399080
:100FE90000AEE0F404255FF53A9000BFE0FE900002
:100FF900AEE0F4042EF53BE538B539058538378080
:1010090003120DE485372B752A000210BD9000E606
:10101900E0D3955F5011E537900246126BD6E0F5A3
:101029002B752A000210BD9000AFE0D3955F5043A5
:10103900E537900226126BD6E0F538E5379002467F
:10104900126BD6E0F5399000AFE0F404255FF53A6C
:101059009000E6E0FE9000AFE0F4042EF53BE538A1
:10106900B539058538378003120DE485372B752A84
:10107900008041E537900206126BD6E0F538E53776
:10108900900226126BD6E0F5399000BFE0F40425F2
:101099005FF53A9000AFE0FE9000BFE0F4042EF552
:1010A9003BE538B539058538378003120DE48537B6
:1010B9002B752A00229000F7E0F53C753F11755A0F
:1010C90002755B00AE52AF53E53C75F00FA4FDAC61
:1010D900F0EDD39FEC9E4021E53C8E048F05FF1275
:1010E9006B94ED75F010A4FFAEF0E55F75F0118417
:1010F900FD7C00ED2FF53D800EE55F75F01184FF55
:101109007E00EF24F0F53D853D37E55F75F01184EC
:10111900AFF07E008F3A120D6A85373EAE52AF535B
:101129009000F7E075F00FA4FDACF0EDD39FEC9EB5
:101139004028755A02755B10853D37120D6A853E48
:1011490038853739AE52AF53E53C8E048F05FF120F
:101159006BBF8D3A853C3B120DE485372975280014
:10116900752B64752A00229000F7E0F53C753F1154
:10117900755A02755B00AE52AF53E53C75F00FA48A
:10118900FDACF0EDD39FEC9E4021E53C8E048F052C
:10119900FF126B94ED75F010A4FFAEF0E56175F0E8
:1011A9001184FD7C00ED2FF53D800EE56175F01190
:1011B90084FF7E00EF24F0F53D853D37E56175F04C
:1011C9001184AFF07E008F3A120D6A85373EAE5218
:1011D900AF539000F7E075F00FA4FDACF0EDD39F8D
:1011E900EC9E4028755A02755B10853D37120D6AD1
:1011F900853E38853739AE52AF53E53C8E048F05AD
:10120900FF126BBF8D3A853C3B120DE4853729757A
:101219002800E56B6017E56BC394FE50109000EB56
:10122900E0B402099000D9E0D3940B50028017AEC4
:1012390028AF29E56B126BA474E78E048F05FF12A2
:101249006B948C288D299000C1E0B40453E55F7537
:10125900F00484FF7E008F37E55F75F00484ADF0FC
:101269007C008D3A753F04755A01755B00E537C3FB
:10127900943F5005120D6A80069001C5E0F537AE1E
:1012890028AF29E537126BA474648E048F05FF1209
:101299006B94AE28AF29EF2DFDEE3CFC8C288D29EF
:1012A900752B64752A002290008CE0B40146E5672D
:1012B90075F00A84FF7E008F37E56775F00A84AD03
:1012C900F07C008D3A753F0A755A05755B00E53764
:1012D900C394115005120D6A8006900597E0F53701
:1012E900AE2AAF2BE5372FFF50010E7464126BE85D
:1012F9008E2A8F2B90008DE0B40146E56875F00ABF
:1013090084FF7E008F37E56875F00A84ADF07C00B4
:101319008D3A753F0A755A05755B6CE537C39411AB
:101329005005120D6A8006900603E0F537AE2AAF24
:101339002BE5372FFF50010E7464126BE88E2A8F4C
:101349002B90009CE0B40249E56AC3944175F0050D
:1013590084FF7E008F37E56A75F00584ADF07C0067
:101369008D3A753F05755A06755B00E537C39413C9
:101379005005120D6A8006900699E0F537AE2AAF3E
:101389002BE5372FFF50010E7464126BE88E2A8FFC
:101399002B9000DEE0B40202800302144FE55F7572
:1013A900F01584FF7E008F37E55F75F01584ADF089
:1013B9007C008D3A753F15755A03755BF4E537C3A3
:1013C900940B5005120D6A8006900485E0F537E507
:1013D9003775F0FFA4FFAEF09000DFE08E048F05B3
:1013E900FF126B94ED900079F0E56675F078A4FF33
:1013F900AEF074FF8E048F05FF126B948C5A8D5BCF
:1014090074028C068D071200398F37AC5AAD5B74A4
:1014190004FF126BBF8D3A753F04755A06755B2838
:10142900E537C3941D5005120D6A80069006CBE07E
:10143900F537AE2AAF2BE5372FFF50010E74641232
:101449006BE88E2A8F2B90008BE0B4025DE5617505
:10145900F064A4FFAEF074081200398E5C8F5D74DD
:10146900058E048F05FF126B948D37AE5CAF5D74EA
:10147900058E048F05FF126BBF8D3A753F05755AAE
:1014890005755BDEE537C394135005120D6A8006B6
:10149900900677E0F537AE2AAF2BE5372FFF5001DD
:1014A9000E7464126BE88E2A8F2B9000CDE0703C8D
:1014B900900055E075F00584FF7E008F3790005548
:1014C900E075F00584ADF07C008D3A753F05755ADD
:1014D90005755BC0E537C3941D5005120D6A80067A
:1014E900900663E0F537E537900081F0229000948B
:1014F900E0B401179007D1E0252BFFAE2A50010E69
:101509009000E8E0126BE88E2A8F2B90010CE0B472
:10151900011490010DE0A852B8000495535007E555
:101529005FC39560400280129000B6E0252BFFAEA4
:101539002A50010E8E2A8F2B802F900094E0B4033D
:1015490016A22AB3B350109007D4E0C39405A85249
:10155900B800069553400280109000B6E0252BFF95
:10156900AE2A50010E8E2A8F2B90008EE0B4020213
:1015790080030218F4900091E0602FE567D3944648
:10158900402890001BE0FEA3E0FF9000CCE075F03E
:1015990003A4FDACF0EFD39DEE9C400E9000F0E06B
:1015A900A852B80005D3955350030218F49000C10E
:1015B900E0B40302800302175885615B755A0090F5
:1015C9000098E0A852B800049553500E900099E095
:1015D900A85AB80005D3955B5003021755E5617504
:1015E900F002A4FFAEF074158E048F05FF126B9400
:1015F9008C068D07900616126BCBFEE0FFEE90006D
:1016090090E0FEEF8E0088F0A4FFAEF074648E04C3
:101619008F05FF126B948C5A8D5B900055E075F025
:1016290018A4FFAEF09000D7E08E048F05FF126B6F
:10163900948C068D0790062E126BCBAE5AAF5BE0E9
:10164900126BA474648E048F05FF126B948C5A8DEF
:101659005BE565A85AB80077D3955B4072E565C329
:10166900955BFFE4955AFE8E5A8F5B7428BE000382
:101679009F500C755B28755A00740D900056F0AE9A
:101689005AAF5B900091E0126BA474288E048F0509
:10169900FF126B948C5A8D5BAE28AF29740A8E04A5
:1016A9008F05FF126B948D068C07AC5AAD5BCFCEBC
:1016B900CF120003740A8E048F05FF126B948C5AA3
:1016C9008D5BAE28AF29126BF08E288F29807DE5BE
:1016D90065A85AB80004955B5072AE5AAF5BE565D0
:1016E900126BE88E5A8F5B7428BE00039F500C75ED
:1016F9005B28755A00740D900056F0AE5AAF5B9096
:101709000091E0126BA474288E048F05FF126B946C
:101719008C5A8D5BAE28AF29740A8E048F05FF128F
:101729006B948D068C07AC5AAD5BCFCECF120003FC
:10173900740A8E048F05FF126B948C5A8D5BAE2848
:10174900AF29EF2DFDEE3CFC8C288D290218F49071
:1017590000D9E0855FF0A4FFAEF07405126BA474A4
:10176900071200398E5A8F5B900098E0A852B80092
:101779000495535012900099E075F002A4FDACF065
:10178900EFC39DEE9C40030218F4E55F75F00B84EE
:10179900FF7E00900616126BCBFEE0FFEE900090E4
:1017A900E0FEEF8E0088F0A4FFAEF074648E048F23
:1017B90005FF126B948C5A8D5B900055E075F018FB
:1017C900A4FFAEF09000D7E08E048F05FF126B9452
:1017D9008C068D0790062E126BCBAE5AAF5BE012CA
:1017E9006BA474648E048F05FF126B948C5A8D5B05
:1017F900E565A85AB80077D3955B4072E565C3954E
:101809005BFFE4955AFE8E5A8F5B7428BE00039FD6
:10181900500C755B28755A00740D900056F0AE5A3D
:10182900AF5B900091E0126BA474288E048F05FFC2
:10183900126B948C5A8D5BAE28AF29740A8E048F73
:1018490005FF126B948D068C07AC5AAD5BCFCECFDA
:10185900120003740A8E048F05FF126B948C5A8D43
:101869005BAE28AF29126BF08E288F29807DE56544
:10187900A85AB80004955B5072AE5AAF5BE5651281
:101889006BE88E5A8F5B7428BE00039F500C755B02
:1018990028755A00740D900056F0AE5AAF5B90004F
:1018A90091E0126BA474288E048F05FF126B948C3F
:1018B9005A8D5BAE28AF29740A8E048F05FF126B0F
:1018C900948D068C07AC5AAD5BCFCECF1200037452
:1018D9000A8E048F05FF126B948C5A8D5BAE28AF6C
:1018E90029EF2DFDEE3CFC8C288D29229000ECE09F
:1018F900B4026AE55F75F00884FF7E008F37E55F03
:1019090075F00884ADF07C008D3A753F08755A0171
:10191900755BE0E537C3943F5005120D6A80069068
:101929000285E0F53785372D752C00AE2CAF2DAC2F
:101939002AAD2B12000374648E048F05FF126B9479
:101949008C2C8D2D900089E08C068D07126BA47468
:10195900648E048F05FF126B948C2C8D2DAE28AFED
:1019690029AC2AAD2B12000374648E048F05FF1273
:101979006B948C288D29900089E08C068D07126B59
:10198900A474648E048F05FF126B948C288D29A290
:101999000B401DAE52AF537405BE00039F5002D2D7
:1019A9000BE561D394CC4008D2017411900056F034
:1019B9009000EBE0B402089000D9E0640B6002806B
:1019C90035AE28AF29E56B126BA474E78E048F0539
:1019D900FF126B948C288D299000ECE0B40217AEAD
:1019E9002CAF2DE56B126BA474E78E048F05FF12E3
:1019F9006B948C2C8D2D9000ABE05402601B9000F1
:101A0900A2E0A852B80012D39553400DA20BB3B36C
:101A19005007E561C3949A40028028AE34AF3590EF
:101A290000A0E075F002A4FDACF0EF2DFDEE3CFC4A
:101A390074022DFD50010CE561BC0007D39D4003E4
:101A4900754301856135753400E5437003021B3820
:101A59009000FEE0C395435003021B2A90010EE05B
:101A6900C394025076E56775F00A84FF7E009005FD
:101A790086126BCBE0F55B755A00AE5AAF5B9000EE
:101A8900A1E0126BA474648E048F05FF126B948C11
:101A99005C8D5D9000FEE004C395438C068D0712B2
:101AA9006BA49000FEE08E048F05FF126B948C5C92
:101AB9008D5DAE28AF29EF2DFDEE3CFC8C288D29DC
:101AC9009000ECE0B40212AE2CAF2DAA5CAB5DEF36
:101AD9002BFBEE3AFA8A2C8B2D80469000FEE0040F
:101AE900C39543854BF0A4FFAEF09000FEE08E0451
:101AF9008F05FF126B948C5C8D5DAE28AF29EF2D9D
:101B0900FDEE3CFC8C288D299000ECE0B40212AE6D
:101B19002CAF2DAA5CAB5DEF2BFBEE3AFA8A2C8B2E
:101B29002D05439000FEE0C3954350037543009093
:101B390000ABE05401601B90009FE0A852B800126E
:101B4900D39553400DA20BB3B35007E55FC394CCB3
:101B59004002802590009DE075F003A4FFAEF0E5FA
:101B6900402FFF50010E74032FFF50010EE55FBE99
:101B79000007D39F4003754401855F40E544700326
:101B8900021C6B9000FFE0C395445003021C5D905A
:101B9900010EE0C394025076E56775F00A84FF7E72
:101BA90000900586126BCBE0F55B755A00AE5AAF13
:101BB9005B90009EE0126BA474648E048F05FF1283
:101BC9006B948C5C8D5D9000FFE004C395448C069A
:101BD9008D07126BA49000FFE08E048F05FF126B36
:101BE900948C5C8D5DAE28AF29EF2DFDEE3CFC8C0D
:101BF900288D299000ECE0B40212AE2CAF2DAA5C1E
:101C0900AB5DEF2BFBEE3AFA8A2C8B2D80469000C8
:101C1900FFE004C39544854CF0A4FFAEF09000FFAB
:101C2900E08E048F05FF126B948C5C8D5DAE28AF3E
:101C390029EF2DFDEE3CFC8C288D299000ECE0B4B9
:101C49000212AE2CAF2DAA5CAB5DEF2BFBEE3AFA7C
:101C59008A2C8B2D05449000FFE0C39544500375F1
:101C69004400900101E02529FFAE2850010E8E287D
:101C79008F299000B0E0A828B80004952950099050
:101C890000B0E0F5297528009000ECE0B4020D9051
:101C990000B0E0A82CB80006952D400280099000FC
:101CA900B0E0F52D752C00229000ECE0B401028023
:101CB90003021DBCA20BB35003021DBA9000B7E08A
:101CC900B40168AE28AF29AC52AD53120003743C7D
:101CD9008E048F05FF126B949000C7E0BC00109D25
:101CE900400D9000C9E0A828B8000495295002D2F7
:101CF90002AE28AF29AC52AD53120003743C8E04D6
:101D09008F05FF126B949000C7E0C3940ABC0015BD
:101D1900D39D40119000C9E0C39405A828B80005D7
:101D2900D3952950028002C2028068AE28AF29AC3F
:101D390052AD5312000374788E048F05FF126B9411
:101D49009000C7E0BC00109D400D9000C9E0A82894
:101D5900B8000495295004D2028038AE28AF29ACC6
:101D690052AD5312000374788E048F05FF126B94E1
:101D79009000C7E0C3940ABC0015D39D40119000A0
:101D8900C9E0C39405A828B80005D3952950028055
:101D990002C202A202B34019AE28AF299000C8E0DE
:101DA900126BA474648E048F05FF126B948C288DBA
:101DB900298002C202A200B34006A201B3B35009AE
:101DC900900021E4F0A3F08024AE28AF297400D359
:101DD9009F74019E400C900021E528F0A3E529F0AD
:101DE900800B74FF900021F8E4F0E8A3F09000CE96
:101DF900E0D39402400C9000B9E07006A20BB3B393
:101E09004002801AAE28AF297402126BA48E288F63
:101E190029AE2CAF2D7402126BA48E2C8F2D90003D
:101E2900B7E0B4011AAE28AF297402126BA48E2848
:101E39008F29AE2CAF2D7402126BA48E2C8F2DAE70
:101E490028AF29745E126BA4740A8E048F05FF12E1
:101E59006B948C288D299000ECE0B40217AE2CAF5E
:101E69002D745E126BA4740A8E048F05FF126B9495
:101E79008C2C8D2DAE28AF297402BE000AD39F4049
:101E890006752902752800AE2CAF2D7402BE000A12
:101E9900D39F4006752D02752C0090001FE528F090
:101EA900A3E529F022900055E0900386126BD6E055
:101EB900F541754264900055E0FE9000C2E0D39E62
:101EC9004037E55F75F00884FF7E008F37E55F7561
:101ED900F00884ADF07C008D3A753F08755A03759A
:101EE9005B96E537C3941F5005120D6A800690046E
:101EF9003BE0F5378537428035E55F75F00884FFAB
:101F09007E008F37E55F75F00884ADF07C008D3A6F
:101F1900753F08755A03755BB6E537C3941F5005BD
:101F2900120D6A800690045BE0F5378537422290EE
:101F390000F8E0F53C753F11755A04755B00AE5227
:101F4900AF53E53C75F00FA4FDACF0EDD39FEC9ECB
:101F59004021E53C8E048F05FF126B94ED75F0105E
:101F6900A4FFAEF0E55F75F01184FD7C00ED2FF55F
:101F79003D800EE55F75F01184FF7E00EF24F0F5DA
:101F89003D853D37E55F75F01184AFF07E008F3AEE
:101F9900120D6A85373EAE52AF539000F8E075F0E6
:101FA9000FA4FDACF0EDD39FEC9E4028755A047543
:101FB9005B10853D37120D6A853E38853739AE523B
:101FC900AF53E53C8E048F05FF126BBF8D3A853CFC
:101FD9003B120DE4853741754264229000F8E0F523
:101FE9003C753F11755A04755B00AE52AF53E53C21
:101FF90075F00FA4FDACF0EDD39FEC9E4021E53CBC
:102009008E048F05FF126B94ED75F010A4FFAEF0EE
:10201900E56175F01184FD7C00ED2FF53D800EE53D
:102029006175F01184FF7E00EF24F0F53D853D37A1
:10203900E56175F01184AFF07E008F3A120D6A8563
:10204900373EAE52AF539000F8E075F00FA4FDACE7
:10205900F0EDD39FEC9E4028755A04755B10853DC1
:1020690037120D6A853E38853739AE52AF53E53C94
:102079008E048F05FF126BBF8D3A853C3B120DE430
:102089008537417542649000C1E0B40479900055E8
:10209900E0FE9000C2E0D39E4037E55F75F008840A
:1020A900FF7E008F37E55F75F00884ADF07C008D09
:1020B9003A753F08755A03755B96E537C3941F5007
:1020C90005120D6A800690043BE0F537853742809A
:1020D90035E55F75F00884FF7E008F37E55F75F0A1
:1020E9000884ADF07C008D3A753F08755A03755B1D
:1020F900B6E537C3941F5005120D6A800690045B3C
:10210900E0F5378537422290008CE0B4013BE56762
:1021190075F00A84FF7E008F37E56775F00A84AD94
:10212900F07C008D3A753F0A755A05755B12E537E3
:10213900C394115005120D6A80069005A9E0F53780
:10214900E5422537C39464F54290008DE0B4013B24
:10215900E56875F00A84FF7E008F37E56875F00A37
:1021690084ADF07C008D3A753F0A755A05755B7E22
:10217900E537C394115005120D6A8006900615E0E3
:10218900F537E5422537C39464F542E5412542F523
:1021990036900094E0B402109007D0E02536FE9006
:1021A90000E8E0F4042EF5369000EBE0D39401400A
:1021B90040E56BC394E7501D74E7C3956BFE900728
:1021C900D2E08E00F5F0E884FF7E008F37E53625F2
:1021D90037F536801CE56BC394E7FE9007D2E08E95
:1021E90000F5F0E884FF7E008F37E536C39537F5B3
:1021F90036A20B4006E5412464F536E536D39464EE
:102209004009E536C39464F53680037536009000BD
:10221900C4E0C3953650069000C4E0F53622D200DA
:1022290090007FE0A852B800049553504190007F78
:10223900E0A852B800049553500375360F90007FFB
:10224900E004A852B800049553500375360A90006B
:102259007FE02402A852B80004955350057536054D
:10226900C20090007FE060067409900056F0C23AFF
:102279007E017F009000CAE0126BA49000D9E08E25
:10228900048F05FF126B94E55FBC0017D39D4013C3
:102299009000D3E0B40204D23A8002C200740A90DA
:1022A9000056F09000CBE0C3956750159000DDE033
:1022B900A852B8000495535002C200740B900056FE
:1022C900F0E567C39464501D900123E0600D90010F
:1022D90023E0A852B80006955340028008C2007452
:1022E9000B900056F0A200400375360590010CE0F2
:1022F900B4011490010DE0A852B800049553500799
:10230900E55FC39560400280089000B5E0F536802E
:102319003A900094E0B40306A22AB3B34002802B9A
:102329009007D4E0C39405A852B800049553500C03
:102339009000B5E0F536740C900056F09007D4E0A3
:10234900A852B8000495535002C20085366C90001B
:1023590086E02536FE900055E075F01E84FC7F006E
:10236900EE2CF53622900055E075F00584FF7E00CD
:102379008F37900055E075F00584ADF07C008D3AFB
:10238900753F05755A03755BD69000D7E01475F053
:102399000584FF7E00E537BE00039F5005120D6AD4
:1023A900800BE53790045C126BD6E0F537E5379082
:1023B90007D3F09007D3E0FE9000C6E0C39E500813
:1023C9009000C6E09007D3F022E56775F00A84FF14
:1023D9007E00900586126BCBE0F546E546D3946402
:1023E9004010E546C3946475F00F84FF7E008F4664
:1023F90080037546009000A9E02546F54622900025
:10240900C1E0C3940350269007C0E0FEA3E0FF7427
:1024190004120039E55F126BA4740F8E048F05FF57
:10242900126B949007BEECF0A3EDF080249007C0E6
:10243900E0FEA3E0FF7404120039E561126BA47495
:102449000F8E048F05FF126B949007BEECF0A3ED7D
:10245900F090009CE0B40262E56AC3944175F0050E
:1024690084FF7E008F37E56A75F00584ADF07C0046
:102479008D3A753F05755A06755B14E537C3941790
:102489005005120D6A80069006ADE0F5379007BE3B
:10249900E0FEA3E0FF740A8E048F05FF126B94E53A
:1024A900378C068D07126BA4740A8E048F05FF12F0
:1024B9006B949007BEECF0A3EDF09007BEE0FEA38D
:1024C900E0FF9007C4E0FCA3E0FDEDD39FEC9E4044
:1024D9000F9007C4E0F8A3E09007BEC8F0A3C8F0C6
:1024E900229006CDE090386BF8282873804C8553EC
:1024F9007380479000D9E0855FF0A4FFAEF07408BF
:102509001200398F738033856173802E85677380DC
:10251900298568738024856973801F856A73801A89
:10252900856B7380158566738010856573800B854F
:0A2539006C738006900022E0F57339
:10386B000224F50224F70224FC022510022515027E
:10387B00251A02251F02252402252902252E0225A1
:07388B003302253802253D40
:102543009006CEE0FE9006CFE0D39E404B9006CDA2
:10255300E0B404189006CFE0C395735002D22B90D9
:1025630006CEE0D395734002C22B802A9006CEE0BC
:10257300C3957350099006CFE0D395735002800240
:10258300D22B9006CEE0D3957350099006CFE0C3CB
:1025930095735002C22B802A9006CEE0D3957340E8
:1025A300099006CFE0C3957340028002C22B9006C8
:1025B300CEE0C3957340099006CFE0D395734002F4
:1025C300D22B229006D1E0903892F8282873804CC1
:1025D30085537380479000D9E0855FF0A4FFAEF088
:1025E30074081200398F738033856173802E856779
:1025F3007380298568738024856973801F856A7356
:10260300801A856B7380158566738010856573806A
:0C2613000B856C738006900022E0F573CC
:103892000225D10225D30225D80225EC0225F10208
:1038A20025F60225FB02260002260502260A02262A
:0738B2000F02261402261983
:10261F009006D2E0FE9006D3E0D39E405F9006D1A5
:10262F00E0B404189006D3E0C395735002D22C90F7
:10263F0006D2E0D395734002C22C803E9006D2E0C2
:10264F00C3957350099006D3E0D39573500280025F
:10265F00D22C9006D2E0D3957350099006D3E0C3E5
:10266F0095735002C22C9006D1E0B401099000E599
:10267F00E0D3956150028002C22C802A9006D2E0EE
:10268F00D3957340099006D3E0C39573400280023F
:10269F00C22C9006D2E0C3957340099006D3E0D3C5
:1026AF0095734002D22C229006D5E09038B9F828C5
:1026BF002873804C85537380479000D9E0855FF075
:1026CF00A4FFAEF074081200398F738033856173E5
:1026DF00802E856773802985687380248569738050
:1026EF001F856A73801A856B7380158566738010DA
:1026FF00856573800B856C738006900022E0F573FF
:1038B9000226C10226C30226C80226DC0226E1022C
:1038C90026E60226EB0226F00226F50226FA022651
:0738D900FF0227040227098A
:10270F009006D6E0FE9006D7E0D39E404B9006D5BC
:10271F00E0B404189006D7E0C395735002D22D9001
:10272F0006D6E0D395734002C22D802A9006D6E0DC
:10273F00C3957350099006D7E0D39573500280026A
:10274F00D22D9006D6E0D3957350099006D7E0C3EB
:10275F0095735002C22D802A9006D6E0D395734010
:10276F00099006D7E0C3957340028002C22D9006F0
:10277F00D6E0C3957340099006D7E0D39573400216
:10278F00D22D229006D9E09038E0F8282873804C9B
:10279F0085537380479000D9E0855FF0A4FFAEF0BA
:1027AF0074081200398F738033856173802E8567AB
:1027BF007380298568738024856973801F856A7388
:1027CF00801A856B7380158566738010856573809D
:0C27DF000B856C738006900022E0F573FF
:1038E00002279D02279F0227A40227B80227BD02B4
:1038F00027C20227C70227CC0227D10227D60227D8
:07390000DB0227E00227E5CE
:1027EB009006DAE0FE9006DBE0D39E404B9006D9D4
:1027FB00E0B404189006DBE0C395735002D22E9020
:10280B0006DAE0D395734002C22E802A9006DAE0F6
:10281B00C3957350099006DBE0D395735002800289
:10282B00D22E9006DAE0D3957350099006DBE0C305
:10283B0095735002C22E802A9006DAE0D39573402E
:10284B00099006DBE0C3957340028002C22E90060E
:10285B00DAE0C3957340099006DBE0D39573400231
:10286B00D22E229006DDE0903907F8282873804C91
:10287B0085537380479000D9E0855FF0A4FFAEF0DD
:10288B0074081200398F738033856173802E8567CE
:10289B007380298568738024856973801F856A73AB
:1028AB00801A856B738015856673801085657380C0
:0C28BB000B856C738006900022E0F57322
:1039070002287902287B022880022894022899023B
:10391700289E0228A30228A80228AD0228B202285E
:07392700B70228BC0228C111
:1028C7009006DEE0FE9006DFE0D39E404B9006DDEB
:1028D700E0B404189006DFE0C395735002D22F903E
:1028E70006DEE0D395734002C22F802A9006DEE011
:1028F700C3957350099006DFE0D3957350028002A9
:10290700D22F9006DEE0D3957350099006DFE0C31F
:1029170095735002C22F802A9006DEE0D39573404C
:10292700099006DFE0C3957340028002C22F90062C
:10293700DEE0C3957340099006DFE0D3957340024C
:10294700D22F229006E1E090392EF8282873804C88
:1029570085537380479000D9E0855FF0A4FFAEF000
:1029670074081200398F738033856173802E8567F1
:102977007380298568738024856973801F856A73CE
:10298700801A856B738015856673801085657380E3
:0C2997000B856C738006900022E0F57345
:10392E0002295502295702295C02297002297502C3
:10393E00297A02297F02298402298902298E0229E5
:07394E009302299802299D54
:1029A3009006E2E0FE9006E3E0D39E404B9006E102
:1029B300E0B404189006E3E0C395735002D230905C
:1029C30006E2E0D395734002C230802A9006E2E02B
:1029D300C3957350099006E3E0D3957350028002C8
:1029E300D2309006E2E0D3957350099006E3E0C33A
:1029F30095735002C230802A9006E2E0D39573406B
:102A0300099006E3E0C3957340028002C23090064A
:102A1300E2E0C3957340099006E3E0D39573400267
:102A2300D230229006E5E0903955F8282873804C7F
:102A330085537380479000D9E0855FF0A4FFAEF023
:102A430074081200398F738033856173802E856714
:102A53007380298568738024856973801F856A73F1
:102A6300801A856B73801585667380108565738006
:0C2A73000B856C738006900022E0F57368
:10395500022A31022A33022A38022A4C022A51024B
:103965002A56022A5B022A60022A65022A6A022A6C
:073975006F022A74022A7997
:102A7F009006E6E0FE9006E7E0D39E404B9006E519
:102A8F00E0B404189006E7E0C395735002D231907A
:102A9F0006E6E0D395734002C231802A9006E6E045
:102AAF00C3957350099006E7E0D3957350028002E7
:102ABF00D2319006E6E0D3957350099006E7E0C354
:102ACF0095735002C231802A9006E6E0D395734089
:102ADF00099006E7E0C3957340028002C231900669
:102AEF00E6E0C3957340099006E7E0D39573400283
:102AFF00D231229006E9E090397CF8282873804C77
:102B0F0085537380479000D9E0855FF0A4FFAEF046
:102B1F0074081200398F738033856173802E856737
:102B2F007380298568738024856973801F856A7314
:102B3F00801A856B73801585667380108565738029
:0C2B4F000B856C738006900022E0F5738B
:10397C00022B0D022B0F022B14022B28022B2D02D3
:10398C002B32022B37022B3C022B41022B46022BF3
:07399C004B022B50022B55DA
:102B5B009006EAE0FE9006EBE0D39E404B9006E930
:102B6B00E0B404189006EBE0C395735002D2329098
:102B7B0006EAE0D395734002C232802A9006EAE05F
:102B8B00C3957350099006EBE0D395735002800206
:102B9B00D2329006EAE0D3957350099006EBE0C36E
:102BAB0095735002C232802A9006EAE0D3957340A7
:102BBB00099006EBE0C3957340028002C232900687
:102BCB00EAE0C3957340099006EBE0D3957340029E
:102BDB00D232229006EDE09039A3F8282873804C6E
:102BEB0085537380479000D9E0855FF0A4FFAEF06A
:102BFB0074081200398F738033856173802E85675B
:102C0B007380298568738024856973801F856A7337
:102C1B00801A856B7380158566738010856573804C
:0C2C2B000B856C738006900022E0F573AE
:1039A300022BE9022BEB022BF0022C04022C09025E
:1039B3002C0E022C13022C18022C1D022C22022C7A
:0739C30027022C2C022C311D
:102C37009006EEE0FE9006EFE0D39E404B9006ED47
:102C4700E0B404189006EFE0C395735002D23390B6
:102C570006EEE0D395734002C233802A9006EEE079
:102C6700C3957350099006EFE0D395735002800225
:102C7700D2339006EEE0D3957350099006EFE0C388
:102C870095735002C233802A9006EEE0D3957340C5
:102C9700099006EFE0C3957340028002C2339006A5
:102CA700EEE0C3957340099006EFE0D395734002B9
:102CB700D233229006F1E09039CAF8282873804C65
:102CC70085537380479000D9E0855FF0A4FFAEF08D
:102CD70074081200398F738033856173802E85677E
:102CE7007380298568738024856973801F856A735B
:102CF700801A856B73801585667380108565738070
:0C2D07000B856C738006900022E0F573D1
:1039CA00022CC5022CC7022CCC022CE0022CE502E8
:1039DA002CEA022CEF022CF4022CF9022CFE022D06
:0739EA0003022D08022D0D60
:102D13009006F2E0FE9006F3E0D39E404B9006F15E
:102D2300E0B404189006F3E0C395735002D23490D4
:102D330006F2E0D395734002C234802A9006F2E093
:102D4300C3957350099006F3E0D395735002800244
:102D5300D2349006F2E0D3957350099006F3E0C3A2
:102D630095735002C234802A9006F2E0D3957340E3
:102D7300099006F3E0C3957340028002C2349006C3
:102D8300F2E0C3957340099006F3E0D395734002D4
:102D9300D23422AE2EAF2F74F5D39F74019E400818
:102DA300782E126BF8022EB0752F01752E00AE52DD
:102DB300AF53E546BE000DD39F40099000BBE0D35F
:102DC300954740028023754700E546C39553F57345
:102DD3009000BEE0D395454008E5452573F5458051
:102DE300069000BEE0F54580020547900097E0D3CA
:102DF3009561401CE55FC395604015AE52AF53E546
:102E030046BE00039F50099000BCE0D395484002A2
:102E1300806E9007D7E0A852B8000495535003750D
:102E23004A009007D7E0A852B8000BD39553400649
:102E3300E5539007D7F0E54A7041E553C39546F54E
:102E430073E573D3940540037573059000BDE0C328
:102E530095455007E573C3954540028009E545C391
:102E63009573F54580069000BDE0F5459000BDE003
:102E7300D3954540069000BDE0F5457548008002B6
:102E83000548E54A7016900097E0C39561500DE53B
:102E9300462405A852B8000695534002800F9000BF
:102EA300AAE0F545754A0174789007D7F022AE2E53
:102EB300AF2F74E9D39F74039E4008782E126BF8EA
:102EC30002304F752F01752E00754532A235402A09
:102ED3007545199000AAE075F002A4FFAEF0E5472E
:102EE300BE0006D39F4002D2350547754A03747866
:102EF3009007D7F075490002303EAE52AF53E54616
:102F03006F4E700302303EE546BE000DD39F40096D
:102F13009000BBE0D395474002800F754700E54A18
:102F2300C394035003754519800DE546C39553F5C6
:102F330073E5472573F547900097E0D39561400EFD
:102F43009007D7E0A852B80007D395534002800CEE
:102F530005499000AAE0B54903754A00E54AB40360
:102F630006A20BB3B34002800A0549E549B43C030A
:102F7300754A02E54AB402299007D7E0A852B8007F
:102F83000ED395534009E5539007D7F07549009048
:102F93000097E0C39561500975490074789007D78D
:102FA300F0E54A705A900097E0D39561401CE55FC5
:102FB300C395604015AE52AF53E546BE00039F5024
:102FC300099000BCE0D3954840028008754800751D
:102FD300454B8028E553C39546F573E573D39405B4
:102FE3004003757305900097E0D395614008E54869
:102FF3002573F5488006E5482406F548754900E53C
:103003004A7016900097E0C39561500DE54624057C
:10301300A852B80006955340028003754A01E54A59
:10302300B4011875451905499000AAE0B54906751C
:103033004A0275490074789007D7F0E54575F00AA0
:10304300A4FFAEF09007C8EEF0A3EFF022E56F9077
:1030530039F1F828287390008FE0700302327790DB
:1030630000C5E0B401028003023192900053E0B541
:103073005E02800302318F7E017F00E5BE126BA4E6
:10308300E5BD2FFF50010E8E5A8F5B7410126BA497
:1030930090007EE08E048F05FF126B949007CCECBA
:1030A300F0A3EDF074FFBC00039D500B74FF900779
:1030B300CCF8E4F0E8A3F0E56B600FE56BC394FE96
:1030C30050089000EBE06402600280649000D9E055
:1030D300B40B1F9007CCE0FEA3E0FF74E7126BA4D0
:1030E300E56B8E048F05FF126B949007CCECF0A375
:1030F300EDF09000D9E0D3940B40089000C1E06458
:10310300046002802B9007CCE0FEA3E0FF9007CE83
:10311300E0FCA3E0FDEFD39DEE9C400D126BF0901D
:1031230007CCEEF0A3EFF080079007CCE4F0A3F018
:1031330090008FE0B4021E9007CCE0FEA3E0FF9066
:1031430007D8E02FFF50010E74011200399007CC0D
:10315300EEF0A3EFF09007CCE0FEA3E0FF9007D8DA
:10316300E0BE0008D39F4004D2388002B2389007F3
:10317300CDE09007D8F09000C1E064016006A2386A
:10318300B3B3400280069007CDE0F55F023275D2FB
:10319300387E017F00E5BE126BA4E5BD2FFF500111
:1031A3000E8E5A8F5B7410126BA490007EE08E0417
:1031B3008F05FF126B949007CCECF0A3EDF0E56B59
:1031C300600FE56BC394FE50089000EBE06402606F
:1031D3000280649000D9E0B40B1F9007CCE0FEA3FB
:1031E300E0FF74E7126BA4E56B8E048F05FF126B8F
:1031F300949007CCECF0A3EDF09000D9E0D3940BBE
:1032030040089000C1E064046002802B9007CCE08A
:10321300FEA3E0FF9007CEE0FCA3E0FDEFD39DEE1D
:103223009C400D126BF09007CCEEF0A3EFF08007FB
:103233009007CCE4F0A3F090008FE0B4021E900757
:10324300CCE0FEA3E0FF9007D8E02FFF50010E74FF
:10325300011200399007CCEEF0A3EFF09007CDE018
:103263009007D8F09000C1E0640160069007CDE0BC
:10327300F55F8003755F0090008BE07006756F014A
:1032830002305075BB1802384590008BE070030282
:1032930033FD7E017F00E5BE126BA4E5BD2FFF5019
:1032A300010E8E5A8F5B9000D1E0B4010F7E0F7F29
:1032B300FFAC5AAD5B126BF08E5A8F5B9000F6E059
:1032C300B40245AE5AAF5B90002BE0FCA3E0FDEDEA
:1032D300D39FEC9E400A90002BE55AF0A3E55BF0E8
:1032E300AE5AAF5B90002DE0FCA3E0FDEFD39DEE63
:1032F3009C400A90002DE55AF0A3E55BF0AE5AAF6F
:103303005B74041200398F619000F6E0704CAE5A82
:10331300AF5B90002BE0FCA3E0FDEFD39DEE9C4060
:1033230009126BF08E5A8F5B8006755B00755A002D
:10333300AE5AAF5B7410126BA490007BE08E048FC7
:1033430005FF126B948C5A8D5B74FFBC0009D39DEF
:103353004005855B6180037561FE9000C1E0B401A7
:103363000280030233FBA20BB3B3500E900095E02F
:10337300A852B80005D39553500280719000D2E053
:103383008561F0A4FFAEF074648E048F05FF126BA9
:10339300948C5A8D5BE56B6016E56BC394FE500FFE
:1033A3009000EBE0B402089000D9E0640B60028067
:1033B30017AE5AAF5B74E7126BA4E56B8E048F05EF
:1033C300FF126B948C5A8D5BAE5AAF5B9007CCE0C7
:1033D300FCA3E0FDEDD39FEC9E4005855B5F800B76
:1033E300A238B340069007CDE0F55F800BA238B357
:1033F30040069007CDE0F55F800375610090008E75
:10340300E07006756F0202305075BB1902384590A3
:10341300008EE070030234B2E55ED395514003029F
:1034230034B0900029E0FEA3E0FFE565126BE8905D
:103433000029EEF0A3EFF07E017F00E5BE126BA43E
:10344300E5BD2FFF50010E8E5A8F5B9000FBE0709D
:1034530013740A126BA474518E048F05FF126B94BC
:103463008D658019AE5AAF5B740A126BA48F048EFC
:10347300057E017F95CDCCCD126A928F65E565D32C
:1034830094644003756564900029E0FEA3E0FFE5C2
:10349300652FFF50010E900029EEF0A3EFF090008E
:1034A30092E0048E048F05FF126B948D6580037583
:1034B30065329000DEE07006756F0302305075BB15
:1034C300130238459000DEE0604A7E017F00E5BECE
:1034D300126BA4E5BD2FFF50010E8E5A8F5B74044F
:1034E3001200398F669000E0E08566F0A4FDACF031
:1034F3007464FF126B948D669000DFE08566F0A420
:10350300FFAEF074FF8E048F05FF126B94ED9000F5
:103513007AF0800375660090008CE07006756F0486
:1035230002305075BB1702384590008CE0B401029D
:1035330080030235C07E017F00E5BE126BA4E5BDAA
:103543002FFF50010E8E5A8F5B9007D9E0601990C0
:1035530007D9E01490661812008CE493FC7401936D
:10356300FDEDC39FEC9E400280069007D9E014F066
:103573009007D9E0C394B3501DAE5AAF5B9007D9FF
:10358300E00490661812008CE493FC740193FDEF41
:10359300C39DEE9C400280069007D9E004F090079B
:1035A300D9E0FE9000B2E08E0088F0A4FFAEF07484
:1035B300648E048F05FF126B948D6780037567001B
:1035C30090008DE07006756F0502305075BB1602D2
:1035D300384590008DE0B4010280030236697E0114
:1035E3007F00E5BE126BA4E5BD2FFF50010E8E5A7E
:1035F3008F5B9007DAE060199007DAE01490678236
:1036030012008CE493FC740193FDEDC39FEC9E4088
:103613000280069007DAE014F09007DAE0C394B36F
:10362300501DAE5AAF5B9007DAE004906782120038
:103633008CE493FC740193FDEFC39DEE9C400280E8
:10364300069007DAE004F09007DAE0FE9000B8E0B5
:103653008E0088F0A4FFAEF074648E048F05FF1211
:103663006B948D68800375680075BB1F0238457EB7
:10367300017F00E5BE126BA4E5BD2FFF50010E8E46
:103683005A8F5B7409126BA474E68E048F05FF12C4
:103693006B948D6A900094E07006756F070230504A
:1036A30075BB15023845900094E070030237C47E61
:1036B300017F00E5BE126BA4E5BD2FFF50010E8E06
:1036C3005A8F5B74041200398F69900094E0B4013F
:1036D300159000E8E08569F0A4FFAEF074071200CE
:1036E30039EF9007D1F0900094E0B402159000E810
:1036F300E08569F0A4FFAEF07407120039EF90077C
:10370300D0F0900094E0B4030280030237A7900046
:10371300D5E0701CE569C394195002D22AE569D338
:1037230094644002C22A9000B4E09007D4F080630E
:103733009000B4E070349000E8E08569F0A4FFAE37
:10374300F074FF8E048F05FF126B94ED9007D4F095
:10375300AE52AF53741EBE0006D39F4002D22AE579
:1037630061D394E54002C22A8029E569C3940A50D3
:103773000DAE52AF53741EBE0004D39F500280029D
:10378300D22AE561D394E54002C22A9000B4E090C6
:1037930007D4F09007D4E0C394055006740590074E
:1037A300D4F0C239900094E0B40414E569C39419C9
:1037B3005002D239E569D394324002C239C22A8019
:1037C300037569009000EBE07006756F08023050D6
:1037D30075BB14806D9000EBE060567E017F00E5C1
:1037E300BE126BA4E5BD2FFF50010E8E5A8F5BEF07
:1037F300D39421EE940E4005756BFF8015AE5AAF3E
:103803005B7410126BA474E38E048F05FF126B9428
:103813008D6BE56B75F00BA4FFAEF09000D9E08ED5
:10382300048F05FF126B949007CEECF0A3EDF080AC
:1038330003756B0090008FE0600575BB1A800375FC
:02384300BB18B0
:1039F10002305902328C0234120234C702352C02D1
:0B3A010035D50236720236A90237D814
:05384500056FD2EC222A
:096BD6002582F58250020583229C
:0F008C0025E050020583258250020583F582226C
:106B7300EF2F500205832582F582E5833E2EF583B0
:016B830022EF
:106BE800CFC39FFF50011E22C3EF9DFFEE9CFE22E4
:086BF8000806B600021806228F
:0D6BB200A3E004F07006120049E004F02298
:0E003900048007C3CE13CECF13CFD5E0F6223E
:106A9200BC000FBE0008ED8FF084FFADF022E4FED3
:106AA200FF22BE000DEF60FE54F0606F20E703028C
:106AB2006B48EAC0E0EBC0E078017A0075F001EEC5
:106AC20020E710EF25E0FFEE33FE0AC5F023C5F004
:106AD20030E7F0EA5407F9096A7A007B006001089E
:106AE200C3EC9E40167004ED9F4010ED9FFDEC9E9E
:106AF200FCE5F0CA4ACA03F5F08005E5F003F5F0BB
:106B0200C3EE13FEEF13FFD9D77908CACBCAD8D088
:106B1200EAFEEBFFD0E0FBD0E0FA22EC8FF084FC3F
:106B2200ED54F045F0C48FF084FEEDC454F045F00E
:106B3200C48FF084FDEEC4FE54F02DFFEE540F3CE2
:106B4200FEADF07C0022790078008FF0EC7E082008
:106B5200E70DC3CD33CD33C933C9C833C8DEF084A2
:106B620049F9E5F08FF0BE00E6FD7C00E9FFE8FEA2
:016B72002200
:0E6BA400F88FF0A4FFE5F0CE88F0A42EFE22BC
:10000300EF8DF0A4F9A8F0EF8CF0A428F8EE8DF0B2
:06001300A428FEE9FF2213
:106B8400600D782B026B8E007830D8FED5E0F822A9
:106B9400EEC0E07E00126A92EFFDEEFCD0E0FE2231
:0C6BBF00EEC0E07E00126A92D0E0FE22E0
:03001B0002001EC2
:0300530002005652
:03009B00020071EF
:03000000026BDFB1
:096BDF0075817575D0000243E9CF
:0B6BCB00E5822FF582E5833EF5832272
:0A0049000582D5820215831582227C
:10001E00C0E0C0F0C083C082C0D075D0001243973C
:0B002E00D0D0D082D083D0F0D0E032E0
:10005600C0E0C0F0C083C082C0D075D00012439A01
:10006600D0D0D082D083D0F0D0E032C0E0C0F0C093
:1000760083C082C0D075D0001243B9D0D0D082D010
:0600860083D0F0D0E0324F
:00000001FF
